:020000040800F2
:10000000F8180020D5000008FF1E0008431E000855
:1000100000000000000000000000000000000000E0
:10002000000000000000000000000000B31F0008F6
:100030000000000000000000811F0008DF1F000812
:10004000E7000008E7000008E7000008E7000008F4
:10005000E7000008E700000899090008E700000829
:100060000000000095090008970900080000000042
:10007000E7000008E7000008E700000800000000B3
:10008000E7000008FD1E000800000000192000081D
:1000900000000000E7000008E7000008E700000893
:1000A00000000000B11F0008E7000008E70000089A
:1000B0007523000800000000E700000800000000B1
:1000C0000348854600F04EF80048004789010008C3
:1000D000F81800200448804704480047FEE7FEE780
:1000E000FEE7FEE7FEE7FEE7ED1F0008C10000089F
:1000F00030B50B46014600202022012409E00D46C0
:10010000D5409D4205D31D469540491B2546954047
:1001100040191546521E002DF1DC30BD03460B433D
:100120009B0703D009E008C9121F08C0042AFAD2AD
:1001300003E00B780370401C491C521EF9D2704733
:10014000D2B201E00270401C491EFBD2704700226F
:10015000F6E710B513460A4604461946FFF7F0FFC6
:10016000204610BD064C0125064E05E0E36807CC8D
:100170002B430C3C98471034B442F7D3FFF7A4FF4D
:10018000B0250008D025000870B50125ED06002433
:1001900006E0A0002858A100064A5050601CC4B2D6
:1001A000302CF6DB012040070349886002F058F943
:1001B000002070BD0000002000ED00E000B58FB011
:1001C0002C2104A8FFF7C3FF0020009001900290AB
:1001D00003900F200490FF200130099000200A9026
:1001E0001348008AC004C00C0121C90308430B90C6
:1001F000002005900C90079002200D9000210E9198
:1002000004A801F029F9002801D000BFFEE707206B
:100210000090022001900020029003900121684686
:1002200000F0AAFF002801D000BFFEE70FB000BD1C
:10023000000FFF1FFEB504460D4600270026281BB1
:10024000800A0190281B8005800D009000BF15E0FA
:10025000124A012080022118204600F0A3FC01214F
:1002600009030E4800F01CF88619012109030B4808
:10027000FFF76DFF0120800224187F1C0198874240
:10028000E6D300982118054A204600F08BFC03486D
:10029000009900F005F886193046FEBDE8020020FE
:1002A00010B502460B460021002000BF02E0545C5E
:1002B0002018491C9942FAD310BD0000FEB504462F
:1002C00000250027002002900190009000268A203F
:1002D000005B0C2807D08821085B0123002211460F
:1002E00000F0E4FBFEBD00BFE81C205C0006A91C7A
:1002F000615C09040843691C615C09020843615D93
:10030000084307462D1D3A4800F05AFC0290029817
:10031000C007C00F029002983840002804D1012184
:100320000198084301904DE0E81C205C0006A91CE0
:10033000615C09040843691C615C09020843615D52
:1003400008432C4988612D1D084680691921C9027E
:10035000884204D9022101980843019032E0002626
:1003600011E00120B040384000280BD0B0002249F5
:10037000085820494860B0001F4908581D49886046
:100380000E7002E0761C002EEBD000BF1949886881
:10039000012101F0B5FD002804D004210198084393
:1003A00001900FE0E81C205C0006A91C615C0904B8
:1003B0000843691C615C09020843615D08430D49FB
:1003C000C86000BF00BF0198002802D194200190AE
:1003D00005E01C210748FFF7BAFE012000908821A4
:1003E000085B042201A9009B00F060FB00BF79E7D5
:1003F00000F400088C010020C800002038B5044635
:1004000000200090002501210098084300908821D9
:10041000085B2B460422694600F048FB38BD00000B
:10042000F8B504460020009003250026084800F097
:10043000C7FB054600950098C007C00F00908821B3
:10044000085B33460422694600F030FBF8BD00002B
:1004500000F40008F0B585B00446002500200390A4
:10046000029001900027002600908A20005B082857
:1004700008DA8821085B01230022114600F016FBF0
:1004800005B0F0BD00BFE81C205C0006A91C615C43
:1004900009040843691C615C09020843615D084363
:1004A00003902D1D524841690398814204D00121D7
:1004B00002980843029085E04D484069401C4C4931
:1004C0004861E81C205C0006A91C615C0904084323
:1004D000691C615C09020843615D084301902D1DA0
:1004E0008A20005B461B4248006980194049086128
:1004F000084600698969884204D910210298084396
:1005000002905FE0B007800F002804D020210298FD
:100510000843029056E0611932463648FFF7FEFD67
:10052000B1030A0C32498868324901F009FD0028FC
:1005300006D002200290022102980843029041E076
:100540002B4A926891192A4A90682B4A00F02AFB9C
:1005500031462948FFF7A4FE07460198874202D09A
:10056000082002902EE02248806880192049886087
:10057000084600698969884219D11D4A52681C4B96
:100580009B69D1181A4A5068FFF754FE074618486D
:10059000C068B84208D18020029018480068012144
:1005A00008431649086001E0402002900AE0104923
:1005B0008868012101F0A4FC002802D0FF2001304E
:1005C000009000BF00BF0298002808D00298802841
:1005D00005D0012000901C210548FFF7B8FD8821B7
:1005E000085B042202A9009B00F060FA00BF47E705
:1005F0008C01002068020020E8010020C4000020D7
:10060000F8B50446002500200090002600F02CFDDF
:10061000054600958821085B33460422694600F0B0
:1006200045FAF8BDF0B502460B460021002400252E
:100630000C2B01DA481EF0BD505CFD280BD1481C84
:10064000105CFC2807D1881C105CFB2803D1C81C57
:10065000105CFA2802D00020C043ECE7081DC1B2AC
:10066000181FC3B2481C105C0002565C304305469C
:10067000881CC1B2981EC3B2481C105C0002565CB4
:1006800030431C4E3081881CC1B2981EC3B2A81ED4
:1006900086B2184846814089882811DC0BE008465C
:1006A0004E1CF1B2165C2046671CFCB2114F803F15
:1006B0003E54581EC3B20F484089A042EFDC02E00E
:1006C0000020C043B7E7042B0EDB505C04280BD19D
:1006D000481C105C032807D1881C105C022803D139
:1006E000C81C105C012802D00020C043A3E70020F2
:1006F000A1E700008001002010B51D480068002817
:1007000000D110BD1A4801781A48FFF78BFF002866
:1007100003D0002016490860F3E7174800F038F8C6
:100720001648008881B2164801F0DAFE0020104910
:10073000086014480078C007C00F002815D00020BA
:1007400011498968C908C90001430F4A916000BF77
:1007500000BF00BF0C488068382108400028F8D14D
:100760000A490878012101F06DFB00BFC9E70000CC
:10077000D0000020E812002000010020CC00002062
:10078000A8010020C4000020001002408C010020BD
:1007900010B504468820005B6038030001F000FEBD
:1007A0000604080C101814182046FFF727FE17E05F
:1007B0002046FFF735FE13E02046FFF77FFD0FE0F0
:1007C0002046FFF747FE0BE02046FFF719FF07E042
:1007D0008821085B01230022114600F067F900BF61
:1007E00000BF002010BD0000F8B505460E461746B4
:1007F000012400BF62480078012801D10220F8BD21
:1008000001205F49087000BF00BF5E4949680722A8
:1008100052031140480B5C49096882005B4B9A58AF
:100820001278914244D15849496882009A58126816
:10083000D201D20D91423BD15349096982009A58A5
:1008400012881204120E914232D14F4989688200F7
:100850009A58127991422BD14B49C96882009A5813
:1008600052685201520D914222D147494969820092
:100870009A589268D203D20B914219D142498969A0
:1008800082009A58D268D203D20B914210D13E49CD
:10089000C96982009A58128A92B2914208D13A49A3
:1008A000096A82009A5812699200920C914244D0CF
:1008B00000BF8100354A51580978334A11608100E0
:1008C000324A51580968C901C90D2F4A5160810047
:1008D0002E4A515809880904090E2B4A11618100DA
:1008E0002A4A51580979284A91608100274A51586B
:1008F00049684901490D244AD1608100234A515871
:100900008968C903C90B204A516181001F4A5158A7
:10091000C968C903C90B1C4A916181001B4A51581F
:10092000098A89B2184AD1618100184A5158096967
:100930008900890C144A116200BF00BF7D20C000ED
:1009400000F096F80446002C13D13A46314628466A
:1009500000F04CF87D20C00000F08AF804460C48F6
:100960004069400840000A494861002C01D02046F7
:1009700045E700BF00200249087000BF20463EE75F
:1009800060140020001002400021024010250008E1
:10099000002002407047704710B5082000F070FA40
:1009A00010BD000000200649486006484069042147
:1009B0000843044948610448C106086070470000C4
:1009C0006014002000200240214334120021054A17
:1009D00051600549496902221143034A5161FF21CF
:1009E000016070476014002000200240F7B5054602
:1009F00000202946019B174E766901273E43154F7B
:100A00007E6100BFEFF31086344672B6012A08D12A
:100A1000104E7669D7043E430E4F7E611E680E600D
:100A200012E00FE01E680E601B1D091D461CF0B28F
:100A3000561E864206D1074E76690127FF043E43C3
:100A4000044F7E619042EDDB00BF84F3108800BF4D
:100A5000FEBD000000200240044949690122D20283
:100A60001143024A5161FF2101607047002002409A
:100A700070B5044600F0F2FA051905E000F0EEFA50
:100A8000A84201D3032070BD064800690121090472
:100A90000840000C0028F1D10348024908610020F9
:100AA000F1E700000020024011800000FFB50020A7
:100AB00004240023FD260746401C384DEE55FC2635
:100AC0000746401CEE55FB260746401CEE55FA260D
:100AD0000746401CEE55002901D0A518ACB20546CA
:100AE000471CB8B22D4F7C55FF252D0225402E12F4
:100AF0000546471CB8B2294F7E55FF260136009D9A
:100B00003543EEB20546471CB8B2244F7E55FF264A
:100B10000136009D3543FF26360235402E1205462C
:100B2000471CB8B21D4F7E55039DEEB20546471CCB
:100B3000B8B21A4F7E55FF263602039D35402E125D
:100B40000546471CB8B2154F7E55002908D0002332
:100B500004E0CD5CC618114FBD555B1C9342F8D321
:100B60008518A8B204260546471CB8B20B4F7E551F
:100B700003260546471CB8B2084F7E550226054697
:100B8000471CB8B2054F7E5501260546471CB8B232
:100B9000024F7E55024D2860FFBD0000A8010020D5
:100BA000CC00002070B505460E462B4605E01846E1
:100BB00000F006F8044610C21B1DB342F7D370BD07
:100BC0000146086870470000F8B504460E46012744
:100BD000002500BF89480078012801D10220F8BD16
:100BE00001208649087000BF00BF85494968072277
:100BF00052031140480B834909688200824B9A587E
:100C00001278914244D17F49496882009A5812680B
:100C1000D201D20D91423BD17A49096982009A589A
:100C200012881204120E914232D1764989688200EC
:100C30009A58127991422BD17249C96882009A5808
:100C400052685201520D914222D16E494969820087
:100C50009A589268D203D20B914219D16949896995
:100C600082009A58D268D203D20B914210D16549C2
:100C7000C96982009A58128A92B2914208D1614998
:100C8000096A82009A5812699200920C914244D0EB
:100C900000BF81005C4A515809785A4A11608100AE
:100CA000594A51580968C901C90D564A5160810015
:100CB000554A515809880904090E524A11618100A8
:100CC000514A515809794F4A916081004E4A515812
:100CD00049684901490D4B4AD16081004A4A51583F
:100CE0008968C903C90B474A51618100464A515876
:100CF000C968C903C90B434A91618100424A5158EE
:100D0000098A89B23F4AD16181003F4A5158096935
:100D10008900890C3B4A116200BF00BF206801288E
:100D200013D17D20C000FFF7A3FE00285ED1FFF79E
:100D300039FE7D20C000FFF79BFE0746334840691F
:100D4000042188433149486150E02068022823D1BA
:100D50007D20C000FFF78CFE002847D1401E306088
:100D6000656812E02846FFF731FE7D20C000FFF7DE
:100D70007FFE074625484069022188432349486190
:100D8000002F01D0356006E08035A068C0016168A1
:100D90004018A842E6D829E02068032826D17D2003
:100DA000C000FFF765FE002820D1401E3060E568D6
:100DB00015E02846FFF750FE7D20C000FFF758FEE3
:100DC0000746124840690121C90288430F4948611A
:100DD000002F01D0356008E0012000032D182069A4
:100DE0000003E1684018A842E3D800BF00BF00201C
:100DF0000249087000BF3846F1E600006014002088
:100E0000001002400021024010250008002002408E
:100E1000012007494969C2071143054A516111463A
:100E20004969C90FC907002900D000207047000098
:100E300000200240002009494969C90FC90700295B
:100E40000BD00749054A91600649916011464969EE
:100E5000C90FC907002900D00120704700200240B7
:100E600023016745AB89EFCD10B5044601F0F2FAD6
:100E7000002803D101F02EFB01F02EF910BD000077
:100E800010B504460748C0682040002808D005482F
:100E9000C460C460062000F041F92046FFF7E4FF7B
:100EA00010BD00000018024070B503460022CBE0E0
:100EB000012696400C683440002C71D04D68022DFC
:100EC00002D04D68122D15D1D508AE001D46203533
:100ED000A8595507EE0E0F25B5400646AE433046DD
:100EE0005607F60E0D69B5402843D508AD001E46DD
:100EF00020367051186856000325B5400646AE43AB
:100F000030460D79AD07AD0F5600B5402843186047
:100F10004D68012D08D04D68022D05D04D68112D6A
:100F200002D04D68122D18D1986856000325B5409F
:100F30000646AE4330465600CD68B540284398601B
:100F40005868012595400646AE43304610264D6848
:100F500035402D09954028435860D8685600032530
:100F6000B5400646AE43304656008D68B54028432E
:100F7000D860012636074D683540B54263D1354DFE
:100F80009608B600A8599507EE0E0F25B5400646FF
:100F9000AE43304605252D07AB4202D1002506E0C1
:100FA00051E02D4DAB4201D1012500E0022596070D
:100FB000F60EB5402843274D9608B600A851254D9A
:100FC000203528680546A5432846012636044D6885
:100FD0003540B54202D10546254328461D4D2035F2
:100FE000286068680546A5432846012676044D68B2
:100FF0003540B54202D1054625432846154D2035DA
:101000006860144D603D28680546A54328460126C2
:1010100036054D683540B54202D105462543284680
:101020000C4D603D286068680546A54328460126AA
:1010300076054D683540B54202D105462543284620
:10104000044D603D6860521C0D68D540002D00D0F5
:101050002EE770BD6018024000040050014800688F
:1010600070470000EC000020014800687047000055
:10107000000EFF1F03480068034909684018014932
:1010800008607047EC000020F400002010B5002438
:10109000032000F009F8002801D0012401E000F04D
:1010A00033F8204610BD0000F8B50446002513486B
:1010B000006800281ED0114801687D20C000FFF79D
:1010C00017F8074639460E480068FFF711F806463C
:1010D00000F0ACFC00280BD1042C07D200222146E2
:1010E000401E00F03FF80748046004E0012502E0DC
:1010F000012500E001252846F8BD0000F40000208D
:10110000FC000020F000002010B500220121112079
:1011100000F028F8112000F013F810BD0146002956
:1011200009DBCB06DB0E01229A40044B1A60BFF3A9
:101130004F8FBFF36F8F00BF7047000080E100E06A
:101140000146002909DB00BF00BFCB06DB0E0122F0
:101150009A40034B1A6000BF00BF00BF70470000F9
:1011600000E100E070B504460D46164629462046CB
:1011700001F024F970BD000070B504460D46002C46
:1011800001D1012070BD6B480068C007C00FA842A4
:1011900018D2684800684008400028436549086044
:1011A000FFF75CFF064607E0FFF758FF801B624928
:1011B000884201D90320E5E75E480068C007C00FF8
:1011C000A842F1D1022120680840022815D104214B
:1011D00020680840042807D158488068072109037F
:1011E0008843401855498860544880680F21090297
:1011F0008843A1680843514988602078C007C00F20
:10120000002854D06068012808D14C4800680121AA
:101210004904084000282ED10120B3E76068002867
:1012200008D146480068012189020840002822D1DF
:101230000120A7E76068022808D140480068012122
:1012400049060840002816D101209BE76068042861
:1012500008D13A484030C0690221084000280AD12C
:1012600001208FE735484030006A022108400028FD
:1012700001D1012086E731488068C008C00061685C
:1012800008432E498860FFF7E9FE064607E0FFF7AE
:10129000E5FE801B2849884201D9032072E72748D0
:1012A0008068382108406168C9008842EFD1214830
:1012B0000068C007C00FA84218D91E48006840083F
:1012C000400028431B490860FFF7C8FE064607E0B8
:1012D000FFF7C4FE801B1849884201D9032051E75B
:1012E00014480068C007C00FA842F1D1042120684B
:1012F0000840042808D11148806807210903884361
:10130000E16808430D49886000F03AF80B498968A4
:101310000F2212021140090A8900094A515CC906CC
:10132000C90EC8400749086007480068FFF7BCFEBF
:1013300028E700000020024088130000001002404F
:1013400030250008FC000020F00000200148006863
:1013500070470000FC00002000B5FFF7F7FF0649CA
:101360008968072212031140090B8900034A515C66
:10137000C906C90EC84000BD001002407025000813
:10138000F0B585B0142230496846FEF7C7FE2F48F5
:10139000806838210840002817D12C4800680902CD
:1013A0000840C10A01268E402848406807214903A9
:1013B0000840450B042D00D90025A9006A46505865
:1013C0003146FEF795FE04463BE020488068382110
:1013D0000840082801D11E4C33E01C4880683821A1
:1013E000084010281BD11948C068C707FF0F002FFD
:1013F00003D0012F0FD1174C10E01448406807218B
:1014000049030840450B042D00D90025A800694672
:101410000858440002E00498440000BF11E00B4863
:10142000806838210840202801D1840209E007485B
:10143000806838210840182802D10124E40300E024
:101440000024204605B0F0BDFC2400080010024036
:1014500000366E01006CDC02FEB50446002C01D1A2
:101460000120FEBD2078C007C00F00286DD0F548D0
:10147000866838210E40C068C707FF0F102E01D1C3
:10148000012F01D0082E0BD1EE480068012149043C
:10149000084000286CD06068002869D10120E0E78E
:1014A000606800280DD0A068002808D0E5480069D1
:1014B0000C218843A1680843E249086101E001204A
:1014C000CFE700BF012109046068884205D1DD48EB
:1014D00000680843DB49086021E0052109046068D1
:1014E00088420ED1D7480068012189040843D549B4
:1014F000086008460068012109040843D1490860D2
:101500000DE0D0480068012109048843CD490860F6
:1015100008460068012189048843CA49086000BF61
:101520006068002812D0FFF799FD054606E0FFF736
:1015300095FD401BC82801D9032092E7C1480068E7
:101540000121490408400028F1D011E0FFF786FD91
:10155000054606E0FFF782FD401BC82801D903209D
:101560007FE7B84800680121490408400028F1D10C
:10157000022120680840022874D1B24880683821CE
:1015800008400646AF48C068C707FF0F102E01D1BC
:10159000002F01D0002E48D1AA48006801218902FD
:1015A0000840002804D06069002801D1012058E7D4
:1015B000A4484068000C0004E1690843A149486060
:1015C000FFF74CFD054606E0FFF748FD401B0228EB
:1015D00001D9032045E79B480068012189020840A2
:1015E0000028F1D0002E18D1964800680721C902C2
:1015F0008843A169084393490860FFF7C1FE9149F8
:1016000089680F2212021140090A89008E4A515C32
:10161000C906C90EC8408D4908608D480068FFF7AB
:1016200043FD002848D001201BE7606900282AD02C
:10163000844800680721C9028843A1690843814999
:10164000086008460068891508437E490860FFF76E
:1016500005FD054607E0FFF701FD401B022802D902
:101660000320FEE628E0774800680121890208404F
:101670000028F0D073484068000C0004E16908437A
:101680007049486018E06F480068FF2101318843C5
:101690006C490860FFF7E2FC054606E0FFF7DEFC58
:1016A000401B022801D90320DBE6664800680121BF
:1016B000890208400028F1D1082120680840082844
:1016C00049D1604880683821084018280BD15D480E
:1016D0004030006A0221084000283CD0206A0028DF
:1016E00039D10120BDE6206A00281AD05548403083
:1016F000006A01210843534940310862FFF7AEFCFC
:10170000054606E0FFF7AAFC401B022801D903208A
:10171000A7E64C484030006A022108400028F1D07A
:1017200019E048484030006A4008400045494031CF
:101730000862FFF793FC054606E0FFF78FFC401BAD
:10174000022801D903208CE63E484030006A02217D
:1017500008400028F1D104212068084004287BD1EA
:1017600000200190374880683821084020280BD19C
:1017700034484030C0690221084000286DD0E0683C
:1017800000286AD101206CE62E48C06B010F0120B1
:101790008843002810D000BF2A48C06B01210907E8
:1017A00008432849C8630846C06B090408400090F4
:1017B00000BF00BF0120019026480068FF210131D1
:1017C0000840002816D123480068084321490860D2
:1017D000FFF744FC054606E0FFF740FC401B0228EB
:1017E00001D903203DE61B480068FF210131084074
:1017F0000028F1D0E068002817D0032109042069EF
:101800000840002808D10F48006988430121490495
:1018100040180C49086108E00A48006903210904DE
:101820008843216908430749086100BFE06801282F
:1018300014D104484030C0690121084301494031B6
:10184000C86127E00010024030250008FC0000209D
:10185000F00000200070004052E050E0E0680528F1
:101860000CD16F48C069042108436D49C86108461E
:10187000C069012108436A49C8610BE06848C06932
:10188000400840006649C8610846C0690421884391
:101890006349C86100BFE068002812D0FFF7DEFB93
:1018A000054607E0FFF7DAFB401B5E49884201D995
:1018B0000320D6E55A48C069022108400028F1D02B
:1018C00011E0FFF7CBFB054607E0FFF7C7FB401B26
:1018D0005449884201D90320C3E55148C069022117
:1018E00008400028F1D10198012808D14C4840381F
:1018F000C06B01210907884349494039C86300BFCB
:10190000606A002858D0464840388068382108402E
:10191000102875D0606A02284FD1414840380068CD
:101920000121090688433E4940390860FFF796FBCC
:10193000054606E0FFF792FB401B022801D9032071
:101940008FE53748403800680121490608400028E3
:10195000F0D1A06A012800D100BFA06A002806D1FA
:1019600000F018FB3049884201D2012079E52C486B
:101970004038C06840084000A16A084328494039FF
:10198000C860084600680121090608432449403917
:101990000860FFF763FB054606E0FFF75FFB401BAF
:1019A000022801D903205CE51D4840380068012168
:1019B000490608400028F0D030E019484038006857
:1019C0000121090688431649403908600846C06865
:1019D00040084000C860FFF741FB054606E0FFF7FE
:1019E0003DFB401B022801D903203AE50C48403852
:1019F00000680121490608400028F0D10EE0FFE709
:101A0000606A012800D12CE505484038C768F9070D
:101A1000C90FA06A814201D0012022E5002020E503
:101A200040100240881300000024F40070B5044602
:101A30002546681E0949884201D901200CE0681E2C
:101A4000074948610321081F00F0B8FC0020044941
:101A5000886107200861002070BD0000FFFFFF00C3
:101A600000E000E003480069022188430149086161
:101A70007047000000E000E070477047704710B505
:101A800004462068006902210840400800281CD054
:101A90002068C06808404008002816D0481F216808
:101AA000086101202077206880698007800F002866
:101AB00003D02046FFF7E2FF05E0204600F0C3F820
:101AC000204600F0C1F8002020772068006904213A
:101AD0000840800800281DD02068C06808408008A1
:101AE000002817D0C84321680861022020772068A9
:101AF0008069032109020840002803D02046FFF72F
:101B0000BDFF05E0204600F09EF8204600F09CF85E
:101B1000002020772068006908210840C0080028BC
:101B20001CD02068C0680840C008002816D0C843F0
:101B300021680861042020772068C0698007800F31
:101B4000002803D02046FFF799FF05E0204600F06B
:101B50007AF8204600F078F80020207720680069A5
:101B600010210840000900281DD02068C0680840E6
:101B70000009002817D0C843216808610820207791
:101B80002068C069032109020840002803D02046CC
:101B9000FFF774FF05E0204600F055F8204600F0FE
:101BA00053F80020207720680069C007C00F01218A
:101BB0004840484000280CD02068C0680840484091
:101BC0004840002805D0C81E21680861204600F062
:101BD0003CF82068006980210840C00900280BD02B
:101BE0002068C0680840C009002805D0C8432168A3
:101BF00008612046FFF740FF206800694021084047
:101C0000800900280BD02068C0680840800900289F
:101C100005D0C84321680861204600F017F8206805
:101C2000006920210840400900280BD02068C068C6
:101C300008404009002805D0C843216808612046B3
:101C4000FFF71BFF10BD70477047704770470000DB
:101C50000146044A1068044A0A600022014B1A60D7
:101C600070470000F80000207814002010B50949E2
:101C700009682022114020290AD101684968CAB2A6
:101C800005490B680968491C034C21600349CA5483
:101C900010BD000000440040F8000020781400202F
:101CA00010B50446002C01D1012010BDA069002808
:101CB00000D000E000BF4520005D002805D10021D4
:101CC00044200155204600F030F8242145200155DC
:101CD0002068C0680121490388432168C860204604
:101CE00000F03EFA206A002802D0204600F09CF95D
:101CF000206800690121C9028843216808612068C1
:101D0000406908218843216848612068C068012132
:101D1000490308432168C8600020A06420214520B1
:101D20000155462001550020BFE710B5044600F0DC
:101D300097F9012200211C20FFF714FA1C20FFF75D
:101D4000FFF910BDFFB583B004460D4617460020CD
:101D500001904520005D202871D1002D01D0002F79
:101D600002D1012007B0F0BD01210903A06888421B
:101D700008D12069002805D1E807C00F002801D04C
:101D80000120EFE700BF4420005D012801D10220BF
:101D9000E8E701214420015500BF0020A064212173
:101DA00045200155FFF75AF90190278667860121E2
:101DB0000903A068884205D12069002802D10026C5
:101DC000029502E02E46002002901EE00698009048
:101DD000002280212046019B00F094FA002801D0C7
:101DE0000320BFE7002E09D102980088C005C00D6E
:101DF000216848600298801C029003E030782168D6
:101E00004860761C608E401E6086608E0028DDD1A2
:101E100006980090002240212046019B00F072FAB3
:101E2000002801D003209DE720214520015500BF57
:101E300000214420015500BF002093E7FFE7022066
:101E400090E77047F8B506460D46274C012D1CD18A
:101E50000027264800F054F8002801D000BFFEE714
:101E60000120009001226946204800F069F800280E
:101E700001D000BFFEE71D48FEF7A2FE0746781C12
:101E8000002801D100BFFEE700BF00F093F8FFF784
:101E9000E9FD17480068C068FF21013188431449F3
:101EA0000968C8601248006840694008400010494D
:101EB000096848610E480068C068202188430C49C1
:101EC0000968C86020680B49084001214907884219
:101ED00009D1206880F3088800BF6068064908605F
:101EE000084600688047F8BD002C000800F4000890
:101EF0007C1300200000FE2FC000002070477047B8
:101F000030B587B004460D46002006906006400EAE
:101F1000002803D00020C04307B030BDFEF78AFF81
:101F2000022001900294039506A901A8FEF74CFE39
:101F3000002801D000BFFEE7FEF76AFF0020EBE7B4
:101F400070B504460E461546A80000190B49884294
:101F500002D90020C04370BDA007800F002802D026
:101F60000020C043F7E7FEF765FF2A4631462046CA
:101F7000FEF73AFCFEF74CFF0020ECE700000108FA
:101F8000704710B5FFF782F8FEF718F900F0A4F8D3
:101F900010BD000004484068072252031040410B66
:101FA0008800024A1058704700100240902500082F
:101FB000704770471FB50020009001900290039079
:101FC00007200090002001900290039000216846B5
:101FD000FFF7D2F8002801D000BFFEE71FBD10B503
:101FE000FFF748F800F096F810BD00000748406879
:101FF000000C0004012149034018054949680843C1
:1020000002494860C80303498860704700100240D5
:10201000000FFF1F00ED00E010B50248FFF72FFD95
:1020200010BD0000201400204022016A1140002948
:1020300015D00168496992019143426A11430268CF
:10204000516101221203416A914208D10168496934
:10205000032252039143826A11430268516170471F
:1020600008B500BF1A48406B01210843184948636E
:102070000846406BC007C00F009000BF00BF00BF04
:102080000846C06B0121490408431149C86308464A
:10209000C06B012149040840009000BF00BF04202C
:1020A0000C49086002204860012088600220C86056
:1020B0000420086105200007FEF7F6FE0820054908
:1020C00008600420086105200007FEF7EDFE08BD4A
:1020D000001002400C14002010B50C480C49086098
:1020E0007D20C0024860002109488160C160016113
:1020F00081610C214161FFF7D3FD05480068C0688C
:102100002021084302490968C86010BD004400400E
:102110007C13002010B50E480068002816D00D482A
:102120000068401C0B490860084600680A280DD961
:102130000948FFF78DFD094908600846016806480F
:10214000006800F0B7F900200149086010BD0000E8
:10215000D8000020DC000020E4000020E000002087
:10216000FEB5044620680069012149038843E168FF
:102170000843216808612169A06808436169084330
:1021800002902068C0685E490840029908432168AF
:10219000C860E0690290206840690121C902884353
:1021A00002990843216848612068406903210902B7
:1021B0008843A1690843216848610121C902E06997
:1021C00088424ED1FFF7C8F80546626851001922CF
:1021D0006A431046FDF78CFF06466421FDF788FF31
:1021E00007016268510019226A431046FDF780FF1B
:1021F00006466268510019226A431046FDF778FFCF
:1022000064210090FDF774FF64214843301AC00038
:1022100032300190FDF76CFFF821084040003F1874
:102220006268510019226A431046FDF761FF0646B5
:102230006268510019226A431046FDF759FF642174
:102240000090FDF755FF64214843301AC00032303A
:102250000190FDF74DFF4007400F38182168886056
:102260004CE0FFF779F805466268910019226A434D
:102270001046FDF73DFF06466421FDF739FF0701D3
:102280006268910019226A431046FDF731FF064645
:102290006268910019226A431046FDF729FF642104
:1022A0000090FDF725FF64214843301A00013230C9
:1022B0000190FDF71DFFF02108403F186268910072
:1022C00019226A431046FDF713FF06466268910023
:1022D00019226A431046FDF70BFF64210090FDF7B9
:1022E00007FF64214843301A000132300190FDF7A6
:1022F000FFFE0007000F381821688860FEBD00004F
:10230000F3E9FFFFFFB581B004460D4617460A9E6C
:1023100024E0701C002821D0002E05D0FEF79EFE80
:102320000499401AB04219D92068C068FF21A13130
:1023300088432168C86020684069400840002168DF
:1023400048612021452001554620015500BF00214C
:102350004420015500BF032005B0F0BD206800688F
:102360002840A84201D1012000E00020B842D0D08E
:102370000020F1E710B500F001F810BD10B50548D8
:10238000FFF774FC0020044908600120034908603D
:1023900010BD00007C130020DC000020D8000020CD
:1023A00030B47446641E2578641CAB4204D3635D6C
:1023B0005B00E31830BC18471D46F8E710B500284D
:1023C00019DB1A4A03231B02D21883089B00D25838
:1023D0008307DC0EFF23A3409A438B071B0E840761
:1023E000E40EA3401A43114B032424021B19840852
:1023F000A4001A5118E00E4A03071B0F083B9B0864
:102400009B00D2588307DC0EFF23A3409A438B071F
:102410001B0E8407E40EA3401A43054B0407240F48
:10242000083CA408A4001A5110BD000000E100E01F
:102430001CED00E002E008C8121F08C1002AFAD112
:1024400070477047002001E001C1121F002AFBD134
:10245000704700000148007870470000D400002059
:102460000025002601270024FFF78BFD1048FEF70A
:10247000A7FB05463D4000BF08E00120A0402840E2
:10248000002801D1274603E0601CC4B2012CF4DB14
:1024900000BF0748FEF794FB0646012E03D100213A
:1024A0003846FFF7CFFC01E0FEF726F9FCE7000015
:1024B00000F4000870B505460C462246294603483C
:1024C000FDF72CFE0248046070BD0000E8120020F9
:1024D000D00000200120014908707047D40000207E
:1024E00070B504460D467D23DB002A46214602488E
:1024F000FFF728FC70BD00007C13002000093D00A0
:1025000000127A000024F4004086510100366E016A
:102510001C0FFF1F300FFF1F440FFF1F580FFF1F1F
:102520006C0FFF1F1C0FFF1F1C0FFF1F1C0FFF1F37
:10253000000000000000000000000000000000009B
:10254000000000000000000000000000000000008B
:102550000100000002000000030000000400000071
:10256000060000000700000008000000090000004D
:10257000000000000000000000000000000000005B
:102580000100000002000000030000000400000041
:1025900000093D0000127A000024F4004086510139
:1025A00000366E0100093D0000093D0000093D00B4
:1025B000D02500080000002000010000342400089D
:1025C000D026000800010020F8170000442400086D
:1025D00000000000000000000000000000000000FB
:1025E00000000000000000000000000000000000EB
:1025F00000000000000000000000000000000000DB
:1026000000000000000000000000000000000000CA
:1026100000000000000000000000000000000000BA
:1026200000000000000000000000000000000000AA
:10263000000000000000000000000000000000009A
:10264000000000000000000000000000000000008A
:10265000000000000000000000000000000000007A
:10266000000000000000000000000000000000006A
:10267000000000000000000000000000000000005A
:10268000000000000000000000000000000000004A
:102690000000000000000000002C00080000000006
:1026A000000000000000000000000000000000002A
:1026B000000000000000000000000000000000001A
:1026C00004000000010000000000000000127A0079
:04F400000100000007
:020000040800F2
:102C0000601A0020D52C0008697C0008A97700080C
:102C100000000000000000000000000000000000B4
:102C2000000000000000000000000000A18C00086F
:102C30000000000000000000358400083193000807
:102C4000E72C0008E72C0008E72C0008E72C000818
:102C5000E72C0008E72C0008C14F0008E72C00080B
:102C6000000000007D4A0008814A000800000000C2
:102C7000E72C0008E72C0008E72C00080000000003
:102C8000E72C0008017A000800000000919300087A
:102C900000000000E72C0008E72C0008E72C0008E3
:102CA0000000000029880008E72C0008E72C000835
:102CB0007D9A000800000000E72C000800000000DA
:102CC0000348854600F0CCFC00480047DD3600088C
:102CD000601A00200448804704480047FEE7FEE7EA
:102CE000FEE7FEE7FEE7FEE73D930008C12C000883
:102CF0000549064A08685043054A8018086040089C
:102D00007047014908607047C00000206D4EC64101
:102D10003930000003460B439B0703D009E008C984
:102D2000121F08C0042AFAD203E00B780370401C7B
:102D3000491C521EF9D27047D2B201E00270401C09
:102D4000491EFBD270470022F6E710B513460A462B
:102D500004461946FFF7F0FF204610BDF8B50246BD
:102D60004A40D40F42004B0052085B089A4202D2FC
:102D70000246084611464A0023D0C30D4A00DDB280
:102D8000120EAD1A202D35DA49020126490AF60540
:102D90008A19002C00D0524220214F1B1146B94005
:102DA0002A411018C20D9A4221D0002C17D0012DB3
:102DB00008DCDA05801AD20F8019D207DBB200F0E6
:102DC0007FFBF8BDDA05801A012340001B06C018FE
:102DD00080185A428018CA0F1043490007E049087A
:102DE000C2071143DA05801A80194008801800F0E4
:102DF0005FFBF8BD61000122511A001BF7E70122B9
:102E0000D2075140AAE70122D2075040A6E7024666
:102E100070B54A40D30FDB0740002DD04A002AD0BE
:102E2000010E140E000212020919400A520A8418F7
:102E3000E50104465443000A120A2E045043A41923
:102E40004219200CC543AA18120C0125AD03521CCF
:102E5000521912047F39240400D0521C104301D4AB
:102E60004000491EC2B20C06C0092018401C400890
:102E7000802A02D003E0002070BD400840000029F5
:102E800000DA0020184370BD70B502464A40D50FE5
:102E900040004A00ED0740085208002814D0002ADC
:102EA00012D0C40DD30D41020120C0055202490ABF
:102EB000520AE41A091812187D34914201D3641C95
:102EC00000E04900002C01DA002070BD002391428F
:102ED00001D3891A0343400849000028F7D100298B
:102EE0000AD0914202D10121C90705E0914201D2E5
:102EF000012101E00121C943E005C018401900F09B
:102F0000D7FA70BDF0B507460846584087B0C00FE5
:102F1000049048000E46590040084908BC1A8841F0
:102F200005D2384631461E4617460B460246580023
:102F3000400810434CD0300D039040055900400D1F
:102F4000490D0590401A0290402872DA18030121B9
:102F5000000B09050843019004980092002805D051
:102F6000019952420020884100920190029840212C
:102F70000A1A0199009800F067FA05460C466B465C
:102F800007CB00F082FAC0197141039A0E0D00239D
:102F9000D71756401A467A40164344D0049A002A5E
:102FA0002DD0029A012A039A15DC1205C01A91410C
:102FB00001263605001C7141D20F059ED2070093F1
:102FC000019202962A46234600F0F8FA07B0F0BDB7
:102FD00038463146FAE71605224A0F46B218C01A9B
:102FE000B74101210905001C4F4100187F411146DE
:102FF00018187941E20F10436D19644113E0E2079C
:103000006D0815436408C2071443039A012612058C
:10301000C01A91413605001C7141CE07400830436B
:103020004908C01851412A46234600F0BAFACDE7B4
:10303000FFE7049801224000C117121A00238B41B8
:1030400004983146C417381AA141EEE730B4012480
:10305000E407634030BC55E730B40124E407614025
:1030600030BC4FE70000E0FFF0B50C465C4085B097
:10307000E40FE40703944C000026640859009446CA
:10308000490802460296224321D062460A431ED0D6
:103090006200570D4A000E032303550D012402461A
:1030A0002C492405781B1B0B360B40182343264361
:1030B000614600901C46501AB44103D30098401C4E
:1030C000009002E0921800985B41002803DA00208B
:1030D000014605B0F0BD00200121090507468646DE
:1030E00011E064461D46141BB54106D36546521BCC
:1030F000B341744607430C43A646CD074008490830
:10310000284392185B4105460D43EAD11046184307
:1031100013D06046194650407140084306D06046BF
:10312000101AB34106D20122002306E00022012337
:10313000DB0702E00122D2435310009874460105D8
:10314000381C6141029C039D0019694100F029FA75
:10315000BFE70000FD0300000122D207002800DBCA
:10316000101A002900DB511A814201D80120704752
:10317000002070470122D207002800DB101A002926
:1031800000DB511A814201D20120704700207047B4
:103190000122D207002800DB101A002900DB511A97
:1031A000814201D301207047002070470122D207DD
:1031B000002800DB101A002900DB511A814201D9D6
:1031C00001207047002070470122D207002800DB51
:1031D000101A002900DB511A814201D101207047E9
:1031E0000020704710B5002904DB0C460121C907F7
:1031F0004042A141002B04DB1C460123DB07524265
:10320000A341801A994101D3012010BD002010BDB7
:1032100010B5002904DB0C460121C9074042A14139
:10322000002B04DB1C460123DB075242A341801A1A
:10323000994101D2012010BD002010BDC217C10F5D
:10324000504010B54018CA079623002100F038F905
:1032500010BD10B500229623114600F031F910BDC3
:10326000C20F410040020123400ADB05D207090ECC
:10327000C0187F2901DA00207047962903DC9623C5
:10328000591AC84001E096398840002AF4D04042DB
:103290007047410040020122400AD205090E801801
:1032A0007F2901DA00207047962903DC9622511A03
:1032B000C840704796398840704700004A000903AB
:1032C0000123090B1B051943094B10B5520D9A42F6
:1032D00001DA002010BD064B34339A4203DC9A1AFF
:1032E00000F0C2F810BD03495118884010BD00001D
:1032F000FF030000CDFBFFFFC20FD20740004008D4
:103300000BD0C10D0723DB01C91840020905400A93
:103310001143C2084007114370470020014670471F
:10332000CB0FDB07490010B5490802460A4307D016
:103330000A0D07240903E401090B121B002A01DC12
:10334000002010BDC900440F0C43C100E018D20595
:10335000801800F0ADF810BD70B50446002903D008
:1033600000202022012310E0002801D00020C043CB
:10337000C046C0460DE02546D5408D4205D30D46DA
:103380009540641B1D46954040191546521E002D60
:10339000F1DC214670BD000070B5002504462E46C4
:1033A000002911D0002C01DA01254442002901DA5C
:1033B000012649422046FFF7CFFFB54200D04042E8
:1033C000002D00D0494270BD002C02DA0121C9074E
:1033D00002E0002C00DD03490846C046C0462146F5
:1033E00070BD0000FFFFFF7FF0B51FB40646002050
:1033F00082B005464024019100901BE001992246CD
:103400000F46304600F030F8049A059B801A994127
:1034100010D310461946224600F016F8361A8F418E
:103420000197224601200021009F00F00DF8381876
:103430004D4100902046641E0028DFDC019B00986F
:103440002946324607B0F0BD10B5202A04DB0146FC
:10345000203A9140002010BD914020239C1A034641
:10346000E3401943904010BD10B5202A04DB084604
:10347000203AD040002110BD0B46D340D04020243C
:10348000A21A91400843194610BD10B5202A06DB48
:10349000CB170846203A1041C1170B4306E00B46F4
:1034A0001341D0402024A21A91400843194610BD70
:1034B000002904DA401C490001D14008400070474F
:1034C00070B40024050C05D11024000402D1002999
:1034D00021D01124050E01D100020834050F01D1BD
:1034E0000001241D850F01D18000A41C002801DBF0
:1034F0004000641C002908D020252E1B0D46F540F5
:10350000A14000D001212943084301061B1B000AEA
:10351000DB1D02D5002070BC7047DB051818801831
:103520000029F8DA401C4900F5D170BC4008400081
:103530007047420005D04200120E52428A4201DB1F
:1035400000207047C9050818704770B5002801DCD5
:10355000002070BD410040020126400AF605090E18
:103560008019CA0701D14000491E4D1000221146A2
:103570003F353346CB409B18D418844201D8001BFA
:103580001A464000491C1729F3DD5100814202D23E
:103590000021C94300E00021E8058018FFF788FFFB
:1035A00070BD10B5002B08DA0024401C6141921850
:1035B0005B411A4301D14008400010BDF0B51FB473
:1035C00082B005460C0003D0084607F0E3FD02E098
:1035D00007F0E0FD20300246009021462846FFF724
:1035E00033FF049B059A04460F46184311430843D2
:1035F00014D0184610431BD0009840210A1A1846D0
:103600000599FFF731FF05460E46009A0599049883
:10361000FFF71AFF084305D0012004E02046394691
:1036200007B0F0BD0020C11705430E432C433743BC
:1036300000990E986305401A7905E40A00220C43AC
:10364000FD0A0A3002D500200146E9E701051019FC
:1036500069410C9C0D9D00196941FFF7A2FFDFE74E
:10366000064C0125064E05E0E36807CC2B430C3CD5
:1036700098471034B442F7D3FFF726FB6CBB000821
:103680008CBB000870B58C180578401C6B075B0F6D
:1036900001D10378401C2A1106D10278401C03E0B6
:1036A00006780E70401C491C5B1EF9D12B0705D40F
:1036B0000023521E0DD40B70491CFAE70378401CFE
:1036C000CB1A921C03E01D780D70491C5B1C521E26
:1036D000F9D5A142D8D3002070BD000080B50020EC
:1036E0000749084A43581350001DC028FAD1012049
:1036F00040070549086007F011FB002080BDC04667
:10370000002C00080000002008ED00E0B0B50A4CD5
:1037100020688168022529438160016901220A43EA
:1037200002618049898A8161412000F057F8206850
:10373000016929430161B0BDB806002070B596B09B
:103740000BAC2C212046FFF7FEFA00250A950995BF
:103750000895079511950E200B900C200D900C9557
:103760001595022614960E950120139001021091D2
:1037700017490968174A0A40C003101812902046DA
:1037800002F0D6FC002800D0FEE70A9509950896BD
:103790000720079007A80124214602F0B5FB002866
:1037A00000D0FEE7A00405906002019001A802F09D
:1037B0000DFB002800D0FEE7E00707490A68024336
:1037C0000A60096801400091009816B070BDC046BB
:1037D000100FFF1FFF1F00003C10024010B50446F1
:1037E00003F010FD0A4800680A49FFF7B5FD604381
:1037F00009494860002088600A68012313430B6070
:10380000064A0B681340012BFBD00860886010BD8E
:10381000D000002040420F0010E000E00100010055
:10382000002904D0024A08CA08C0491EFBD17047CB
:1038300004F8000880B500F059FF80BD80B500F0A5
:1038400071FF80BD10B5324C2078012817D1324865
:1038500002F0CAF93148012101700020207030497E
:103860000A78002A01D0087010BD06F04BF804F069
:1038700093FA03480188491C018005F013FA10BD32
:103880002E090020F0B581B0204C48212046FFF7DA
:103890005AFA1F4D2878012812D11E488021FFF7BF
:1038A00052FA1D4802F0A0F91C48012101700020C5
:1038B00028701B490A78002A05D0087001B0F0BDB5
:1038C000002001B0F0BD06F01DF804F0A1F8154D80
:1038D000154829464CC94CC0CCC9CCC009880180C8
:1038E00005F05EFD07F01EFBA080287801F008FDC2
:1038F000002803D105F038FC05F09AFB00F02AFF00
:1039000001F0E2FC01F01CFC01B0F0BDEC0700206E
:103910002A10002014130020AC0600202C100020D8
:1039200028100020D40F0020F40F00200348017855
:10393000002901D0491E01707047C046CC0000200C
:10394000F0B583B002930127082900D2CBE10546E8
:10395000E8480078002800D1C5E10E4605F0ACFF2C
:10396000E54802F041F9288870380D2800D9B5E102
:103970004000C04678448088400087440D00AF0175
:103980001101AF012C01AF014701AF016101AF018E
:10399000AF017B01AF019501B01E0621FFF7FCFCD2
:1039A0000190082E00D299E14A3E0020044605E02D
:1039B000641CE0B20199814200DC8FE103214143A4
:1039C000480028184188062E21D20D2900D98AE105
:1039D0004900C0467944898849008F440D009B0006
:1039E000A000A60084014C006400AC00B200B80046
:1039F0006700BE008401C3000079C449087001F06B
:103A00007FFC0028D4D10020C0490870D0E7891E6F
:103A10000A2900D967E149007944898849008F441F
:103A20002600620162012A00420062016201620115
:103A300045005D000A008188C08800044018FFF737
:103A400008FCAF49FFF720FAFFF756FC0022AD4B08
:103A5000FFF758FA02460B46FFF754FAFFF72EFC21
:103A6000C0B24000A849085AA4490882A0E70079DA
:103A7000A24908609CE781880806000F00D00F214A
:103A800063209E4A1154CBB26521525C934200D907
:103A90008EE7002A6CD0102A77D30F22974B1A5446
:103AA0000E20585484E70079622135E080880106B1
:103AB000090F00D00F206522904900928854C3B2AC
:103AC0006322895C994200D972E7010656D0102B17
:103AD00060D30F20894988540E205EE08188C08819
:103AE00000044018FFF7B5FB8549FFF7CDF9FFF754
:103AF00003FC0022834BFFF705FA02460B46FFF753
:103B000001FAFFF7DBFBC0B240007F49085A7B494E
:103B100088804DE700796421784A505448E78188CD
:103B2000C088764A9080D18042E78188C088734AF5
:103B3000508191813CE78188C088704A108251820F
:103B400036E781796D4A51720079107230E78179D8
:103B50006A4AD173007990732AE780886621674AA0
:103B6000505225E78179654A5175007910751FE734
:103B70000022624B5A540121195419E700205F4971
:103B8000009BC8540120885412E75C4B1A54501E05
:103B900058540DE759498854401E009A885407E745
:103BA000B01E0621FFF7F8FB082E00D296E0002396
:103BB00052491A4604E0521CD3B2984200DC8DE010
:103BC00003245C436300EB185C880F2CF3D80C19BA
:103BD0001B79A375EFE7B01E0621FFF7DDFB082E6A
:103BE0007CD3002345491A4603E0521CD3B29842C5
:103BF00074DD03245C436300EB185C88052CF4D867
:103C000064000C199B885626A353EEE7B01E0621CC
:103C1000FFF7C2FB082E61D3002338491A4603E0A0
:103C2000521CD3B2984259DD03245C436300EB1865
:103C30005C880F2CF4D80C191B793626A355EFE7B6
:103C4000B01E0621FFF7A8FB082E47D300232B49FF
:103C50001A4603E0521CD3B298423FDD03245C4372
:103C60006300EB185C880F2CF4D80C191B792626FE
:103C7000A355EFE7B01E0621FFF78EFB082E2DD3CC
:103C800000231E491A4603E0521CD3B2984225DD98
:103C900003245C436300EB185C880F2CF4D80C19E8
:103CA0001B796826A355EFE7B01E0621FFF774FBCA
:103CB000082E13D3002311491A4603E0521CD3B235
:103CC00098420BDD03245C436300EB185C880F2CE7
:103CD000F4D80C191B794626A355EFE7074878213D
:103CE000FFF7ACFD0027002002990880384603B09A
:103CF000F0BDC046300C0020AC0600203010002083
:103D0000000020410000E0BFD8000020D40F0020B8
:103D100080B503F0B5FD00F0BDFC024804F03EFCA8
:103D200080BDC046EDAE000810B506F0D5FF0028F6
:103D300004D006F069FE01F02FF810BD07F0BEF8C0
:103D4000054C2068002805D081B2044800F008F82E
:103D50000020206010BDC046B40D0020340D0020AE
:103D6000F0B587B0002800D123E10D46002900D12D
:103D70001FE103460022904E1746049005920395DA
:103D80007624315D0A29104600D988E07944097902
:103D900049008F44050D13181E232E3D43484D0046
:103DA000D85DFD287CD1782000213152012076E0B9
:103DB000D85DFC3841424141480070E0D85DFB28A5
:103DC00034D103206BE0D85DFA384142414188008C
:103DD00065E0D85D7A217052052060E07A20315A82
:103DE000DA5D12025118315288B2772853D300207D
:103DF00052E0D85D7821725A531C7352049BB05420
:103E0000059A7A20305A715A814249D1072046E0FA
:103E1000D85D001F41424141C80040E0D85D032801
:103E200004D109203BE0D85D022837D0002036E0DD
:103E3000D85D0128104632D17A20305A029031469E
:103E400033880025AAB20C2050435C4A12585C4EBD
:103E5000B24202D06D1C9A42F4D11346603B052B4E
:103E600023D801259D4033231D421ED0534A1018EC
:103E700082680E46084602999047039D524B55486A
:103E800001885648026818469047642000F080FF79
:103E90000020049B00E00620059A00E00A2030552F
:103EA0007F1CAF4200D06BE783E0112A0E4615D08D
:103EB000434B9A42039DEBD0404A10184068019052
:103EC00006AB0093304602993E4A019DA8470099EF
:103ED00009883A2915D900203B4B66E0374A10186B
:103EE0004068019006AB009330460299354A019D27
:103EF000A84700990D883A2D12D90020039D324B16
:103F00003EE04D00304B31491960012109023288F1
:103F10000A43DA803049098800291BD004221AE0BC
:103F2000294B188129481860A81D98800122100289
:103F300031880143D980002D15D05D810C3318469E
:103F4000204902922A46FEF7E5FE029A1E4B0C35E6
:103F5000A8B209E00222029552199A80002912D0D3
:103F600018810A2010E00A20039D194919541918D4
:103F7000CA70174A120C8A70154A120A4A70001D3C
:103F8000144908807BE70820019018180D49029D0C
:103F90002A46FEF7BFFE0C4B0198401981B20C4A2D
:103FA0005A525918120C4A80001D0A490880039D74
:103FB00065E707B0F0BDC0468C050020F800002082
:103FC000FFFF0000340C00200C050020FDFCFBFA74
:103FD000040302012C09002010120020B80D00205B
:103FE000F0B5CDB01A9319920D4607462FAC782143
:103FF0002046FEF7A8FE1BA85021FEF7A4FE1E21B6
:104000002046FFF70DFC01210026042D00D205E11A
:10401000B9480078002800D100E105F04DFCB74810
:1040200001F0E2FD3888713800260D28189600D975
:10403000EDE0800002A1085818990E468746C04658
:10404000794000080F420008854000080F42000830
:10405000C74000080F4200080D4100080F42000849
:104060004D4100080F4200080F4200088D41000832
:104070000F420008CD4100080026032D00D9D2E0F0
:104080003046D1E0042D00D2C0E0A81EC10F401878
:10409000401000221146164605E0B61C491CCAB263
:1040A000904200DCB3E05200BA1852880F2AF4D8CC
:1040B0002FAB9A18927DF3B25B001BACE252E21870
:1040C00000235380E9E7042D00D29FE0A81EC10F12
:1040D0004018401000221146164605E0B61C491C47
:1040E000CAB2904200DC92E05200BA185288052A07
:1040F000F4D852002FAB9A185623D25AF3B25B0071
:104100001BACE252E21800235380E7E7042D7DD375
:10411000A81EC10F4018401000221146164604E0A8
:10412000B61C491CCAB2904271DD5200BA185288BE
:104130000F2AF5D82FAB9A183623D25CF3B25B0066
:104140001BACE252E21800235380E9E7042D5DD353
:10415000A81EC10F4018401000221146164604E068
:10416000B61C491CCAB2904251DD5200BA1852889E
:104170000F2AF5D82FAB9A182623D25CF3B25B0036
:104180001BACE252E21800235380E9E7042D3DD333
:10419000A81EC10F4018401000221146164604E028
:1041A000B61C491CCAB2904231DD5200BA1852887E
:1041B0000F2AF5D82FAB9A186823D25CF3B25B00B4
:1041C0001BACE252E21800235380E9E7042D1DD313
:1041D000A81EC10F4018401000221146164604E0E8
:1041E000B61C491CCAB2904211DD5200BA1852885E
:1041F0000F2AF5D82FAB9A184623D25CF3B25B0096
:104200001BACE252E21800235380E9E70E46F6B2F7
:1042100072001BA91998FEF77DFD18991A9806805F
:1042200008464DB0F0BD0120042D00D207E16234F4
:10423000A91ECA0F89184B10012117918D4382497D
:1042400009780F91A1780E912FA98A880D92CA88BA
:104250000C924A890B928A890A9262781592227886
:1042600014920A8A09924A8A08924A7A07920A7A2A
:104270000692CA7B05928A7B0492E2781392A28806
:1042800003924A7D0292097D0191B2498A88129275
:10429000098A119100212F9A10920C460E4616930E
:1042A00003E0B61C8B4200DCC9E04900791849885C
:1042B0001A2D13D10D2900D9BDE0C04679440979E2
:1042C00049008F4406606570B8262B7B8691309C30
:1042D000B8A5F0B240001BA90F9A94E0891E0A29E4
:1042E00000D9A8E07944097949008F4409A4A412AF
:1042F00017A4A4A41C212C00300C0020AC06002024
:10430000F0B240001BA9109A0A520818110C418003
:1043100089E0F0B240001BA9159A74E0F0B24000A9
:104320001BA9149A6FE0F0B240001BA9139A6AE02F
:1043300000204649129B0A889A420FD0891C401CD3
:104340001028F8D109E000204049119B0A889A42C0
:1043500004D0891C401C1028F8D11020401CFEF706
:104360006DFF3F210906FEF752FD3949FEF74FFD6B
:10437000FEF78FFFF1B249001BAA50525118000CF2
:104380004880169B4FE0F0B240001BA90E9A3AE01D
:10439000F0B240001BA90C9A0A5201203043C0B26F
:1043A00040000D9A3EE0F0B240001BA90A9A0A5262
:1043B00001203043C0B240000B9A33E0F0B240001D
:1043C0001BA9089A0A5201203043C0B24000099A42
:1043D00028E0F0B240001BA9069A0A52012030439F
:1043E000C0B24000079A1DE0F0B240001BA9049A39
:1043F0000A5201203043C0B24000059A12E0F0B2E8
:1044000040001BA9039A0A520818002141800AE0C3
:10441000F0B240001BA9019A0A5201203043C0B2F9
:104420004000029A0A52641CE1B28B42179800DDE8
:1044300037E7002035E700221A9919920A80C00751
:1044400000D1E4E60121EBE6D40F0020D8000020E3
:1044500000002041F0B58BB01C4601270026002843
:1044600027D0154605F028FA884801F0BDFB88489A
:10447000007801281DD104F07BFF81780291C1787A
:104480000191017800914678011D03AF2022384642
:10449000FEF740FC30020099401801990902029A87
:1044A000891809040E18284639463246FEF732FCB0
:1044B0000027268038460BB0F0BDC046B0B51C467C
:1044C000154605F0F9F9714801F08EFB384800886F
:1044D000002806D008490A222846FEF71BFC0520C2
:1044E00006E00020A88002206880012028800320A8
:1044F00020800020B0BDC046B4B80008F0B581B03F
:104500001C46064662480078012501281CD10F464A
:1045100005F0D2F95D4801F067FB30887A2802D1B6
:10452000718800290CD0082F0ED109280CD1F088F1
:104530006621BB4A50523F4803210170002503E029
:1045400030793C490870002500202080284601B0C1
:10455000F0BDC04630100020F0B581B01C461546B5
:104560000F4600904A4801210170484801F03CFB89
:1045700005F0C0F905F0A6F904F036FD04F046FD9B
:1045800004F012FA0326304603F010F9032F08D383
:104590000098408806490880802068802E8002208C
:1045A00002E00349002008802080002001B0F0BD17
:1045B0001012002010B500241C801C4800683448EC
:1045C000047005F097F904F029FD6420FFF706F95F
:1045D00004F012FD05F0BEF9032003F0E7F8E12036
:1045E000C000FFF7FBF8204601F01CFB274801F054
:1045F000FBFA0F48012101700E480078032805D10D
:1046000003F064FF142000F0C3FB04E07B48007853
:10461000012104F007F803F09FFF07484088400499
:10462000000C04F0C7F9002010BDC046044400404F
:104630002810002034080020E007002070B51C4638
:104640000125002811D0064605F036F90F4801F083
:10465000CBFA0F480078012807D17588212D08D39F
:1046600000202080202D0FD8002500202080284603
:1046700070BD311D284604F07DFE16480188001DDE
:1046800000F038F8202DEFD9012070BDAC060020D5
:10469000300C002080B582B00C4801900C4800908E
:1046A00003F06EFF401C05D00A48092103F06CFF9F
:1046B00002B080BD0820694604F05CFE0548018810
:1046C000001D00F017F802B080BDC0463130364CF6
:1046D00058656E449C13002080B5012041020248B9
:1046E000016001F043FB80BD880800201848006885
:1046F0007047C04670B582B004460191084D01264E
:104700002846314603F012FB01A92846324603F041
:1047100029FB281D0822214603F024FB02B070BDAE
:1047200080FB000870B582B00D4604460191084E2A
:104730000721304603F0FAFA01A90122304603F0BE
:1047400011FB301DAA08214603F00CFB02B070BD1E
:1047500000F80008F0B583B02848017E002903D096
:1047600027A006F007FDFEE763212D4A515C00916A
:10477000C08A019000242B4F2C4B26460CE0284683
:10478000019A06F0BFFB294BE1188870000A4870B7
:10479000761C029C641C234FA0B281007D5AFF2D21
:1047A00005D17A185288204B9A42204B10D002949F
:1047B000F2B2032454431D55791849880928DED3E1
:1047C00000980228DBD8284606F08CFA0146D6E786
:1047D000002017491D460A5CF3B203245C432A55A6
:1047E0002A190B185B8893701B0A5370001D761CE6
:1047F0001428F0D10F48067003B0F0BDD40F00208C
:10480000556E737570706F7274204441544120521C
:1048100065677320436F6E76657274212100000016
:104820003010002060B90008FFFF000038020020AF
:10483000C8BA000811130020F0B587B005920690A1
:10484000664A1078012802D1022007B0F0BD02911B
:1048500001200490107062480068C00A1C210140C9
:1048600060484158604805680A68D7B25F4E614C9D
:10487000614BBD4230D1150C35404468AC425D4CB3
:104880002AD10469120AD2B294425A4C24D18468C3
:104890004A68D5B2AC42574C1ED1120C544C22403F
:1048A000C4689442534C17D142698C681C40A242A0
:1048B000504C11D18269CC681C40A2424D4C0BD1A6
:1048C000C4690A6995B2AC424A4C05D1120C224027
:1048D000046A9442474C16D007604A8832404260CE
:1048E0004A7802610A798260CA88414D2A40C260D2
:1048F0008A681A404261CA681A4082610A8AC261A3
:10490000498A214001627D20C40001F03DF90194F3
:104910000519049806043948041F2768374005D054
:1049200001F032F9A842F6D3032002E034482060B7
:104930000020059A002F30D1304B186804990843A5
:104940001860EFF31080009072B6002A029F06985C
:1049500009D0012A26D10499C904284B1A680A43B0
:104960001A6039680160009880F3108801F00CF932
:10497000019947182568354005D001F005F9B8427E
:10498000F8D3032002E01E48206000201B4B19686A
:10499000049A91431960002D02D100210F4A117031
:1049A00007B0F0BD511E049AD2040392059A002369
:1049B00002E0001D9542D6D220CF05605B1CDDB21F
:1049C000A942F6D1069038460C4F3F68039A174328
:1049D0000A4A176007460698059AEAE7E812002097
:1049E00004100240E8BA000800210240FF01000064
:1049F000FF070000FF3F0000FFFF010014200240FE
:104A000011800000F0B581B000282DD00446064684
:104A1000483602207070206801684022914301608E
:104A2000134988421AD10127B80312490A68024380
:104A30000A600A6882430A600F48042100F040FFC0
:104A4000052005073902284600F03AFF790228467A
:104A500000F036FFB902284600F032FF0020E06483
:104A60003070707001B0F0BD012001B0F0BDC046E3
:104A7000003800402C100240000400507047000035
:104A800080B50248406C00F089FC80BD38080020E9
:104A9000F0B583B0002823D01446002A20D09023FC
:104AA000BA4A15460293D25A2388CF1A974200DB9E
:104AB0001746B9B201918E26A95B6A18C118104633
:104AC000019AFEF727F9A85BC019A8532088381867
:104AD000401E2080029BE85AC01BE852000401D00F
:104AE00003B0F0BD88200521295499484088083832
:104AF000E85203B0F0BDC046B0B500281BD00C464C
:104B00000D4D0020288002F075FF002813D100F021
:104B10003FFC032804D19D482146FEF793FEB0BD1B
:104B20009A482146FEF7AEFE2880002803D00146B1
:104B3000024806F0DBF9B0BD261200201413002055
:104B4000F0B583B00D46064602A900200880158006
:104B5000002E5CD0002D5AD0019202A800210180C5
:104B60008A4F8822B85C082815D8C0467844007956
:104B7000400087440413171B1F252D364400705C2A
:104B8000AA2831D18E230020F852715C0124BC5434
:104B9000FC52397029E00020B85426E0705C00F027
:104BA0006BF821E0705C00F09FF81DE0705C00F095
:104BB000BBF819E002AA30462946FFF769FF13E067
:104BC000705C8E217B5A5C1C7C52F854062006E0F7
:104BD000705C8E217B5A5C1C7C52F8540720B854C0
:104BE00002E0705C00F0B6F8002002994A1C02A9AD
:104BF0000A8091B2A94206D20028B2D003E0705CCC
:104C000000F0B4F8F1E7019B1988891A198003B004
:104C1000F0BDC046F0B581B0044668460280002A67
:104C200026D08D1800273E4612E08A265748805D20
:104C3000FEF77CFE5548865B012004F0B7F9444836
:104C40004088B1B2FFF758FF68460288002A0FD0AB
:104C500091B2681A6A46FFF773FF06490F5500289C
:104C6000F2D03B4800780328DFD00028DDD0E3E70E
:104C700001B0F0BDB811002010B535490A78002107
:104C8000032A2CD87A44127952009744010811164D
:104C900080220243F0231340B02B14D01FE0802267
:104CA0000243F0231340C02B19D138498C310CE05A
:104CB000F0220240802A12D10AE080220243F0232F
:104CC0001340A02B0BD131498A310207120E0A8002
:104CD0008E212E4A535A5C1C5452D05402218820F3
:104CE0002A4A115410BDC04610B519490B782749FE
:104CF0000A468A32002B05D0032B03D0012B0AD1A0
:104D00000A468C3201231B0244011C400309E318AC
:104D10001488E31813808E228B5A5C1C8C52C85462
:104D2000882003220A5410BD10B5094909780129C9
:104D300004D18C21154A535A1B1853528E21134A01
:104D4000535A5C1C5452D05488200421115410BD75
:104D5000E007002010B58E210C4A535A5C1C5452B7
:104D6000D05488200821115410BDC04610B58823A6
:104D7000064A0021D154552805D18E21535A5C1C76
:104D80005452D0540121084610BDC0464C070020A3
:104D900080B500F0FFFB80BD10B506F07FF803F092
:104DA00003FE0324204602F001FD04F0A3FD04F0FD
:104DB00089FD812041007C48018208492204084B7A
:104DC000084C046043608260C160074901220A8088
:104DD00006490A681221904710BDC04680000403AE
:104DE0000800FF01FDFCFBFA10120020B80D0020A6
:104DF00010B50446CA4800F0F7FE22886A49002030
:104E000048730873C872694B12241C80FD230B7011
:104E1000FC234B70FB238B70FA23CB7008230B71A0
:104E200048718A714872042088730320C873022075
:104E3000087401234B745B4804782046584008727C
:104E4000120A1A43CA71621E944162008A7210BD2E
:104E500070B50446B24800F0C7FE524800780125FC
:104E6000002601283346284605D1514800F04EFA65
:104E700001230340002022884B494E730E73CE72EB
:104E80008B724D7402230B740323CB7304238B7337
:104E90004E7208728A714E7108230B71FA23CB701F
:104EA000FB238B70FC234B70FD230B703F4B1224B4
:104EB0001C80120A2A43CA7170BDC046F0B581B089
:104EC000054604F017FD964800F08EFE3548007840
:104ED0000126002701283846344602D1002400F07C
:104EE00057FE2A88030E30494B73030C0B73030AD9
:104EF000CB7288724E74022008740320C873042099
:104F000088734F720C728A714F7108200871FA20F1
:104F1000C870FB208870FC204870FD200870100AC3
:104F20003043C871204601B0F0BDC04610B50446FC
:104F30007B4800F059FE1B480078012813D11C481B
:104F4000012102F0F3FE1B48072102F0EFFE3220A0
:104F5000FFF71EFFBFF34F8F174818490160BFF3DB
:104F60004F8F00BFFDE722880F49012048730223BD
:104F70000B730323CB7204238B7200244C720872D0
:104F80008A714C710B71FA23CB70FB238B70FC235D
:104F90004B70FD230B70054B0E241C80120A02433C
:104FA000CA7110BD300C00200C0500202C09002017
:104FB00000F4000800F800080CED00E00400FA0519
:104FC00080B5082000F0FCFC80BD0000F0B581B089
:104FD000B94D288A03F0FEFB4F49FDF718FFFEF795
:104FE00058F904464D48007800286CD02E684C488B
:104FF00000F0FAFD30462146FEF7AEF9494DC7B242
:10500000002046490870D5480068C16820229143B5
:10501000C160286808210143296000F0B9F903281C
:1050200001D000F075F902F0EDF83F480068016921
:105030000126B143016103F0B7FC3C48FFF7E2FCF5
:1050400004F066F9FFF748FBFEF760FBB00331465A
:1050500000F09EFE01F0D6FA314800F0C5FDFEF7E3
:105060006DFB05F039FE002824D1A3480078022802
:1050700020D191490968A1421CD000F041F90028D3
:1050800018D100F085F9032814D029480646007885
:10509000401CC0B23946FEF75FF93170002909D0D3
:1050A00004F058FC234801880029A9D07B4805F06A
:1050B0001DFFA5E705F010FE002806D004F04AFC0D
:1050C000032002F073FB01B0F0BD03F0A7FF6420E2
:1050D000FEF784FB03F090FF00F046F904F03AFC81
:1050E000032002F063FBE1208000FEF777FB002045
:1050F00000F098FD03F030FA06F028F80E484088DA
:105100004004000C03F056FC112001010B48FDF790
:105110001AFE01B0F0BDC046000020412C10002056
:10512000AC0600200C180240B8060020C011002078
:105130001212002026120020E0070020A8100020F4
:10514000F0B581B000F024F904466A4D6878000794
:10515000400F04D003F05EFA002C0AD133E003F0D4
:1051600051FA6548007800F0CBF8002827D0002CD1
:1051700029D04A4E4A483060032C1BD1B471032019
:10518000B08066204C490D5A4E480088FEF761F801
:105190000446A800FEF752F801462046FDF774FECB
:1051A0004749FDF734FEFEF75BF8F071000A3072F4
:1051B000092064E0B471022C1CD046201BE00020C2
:1051C000A880002CD5D135486E2101706221017173
:1051D000A988418033490978002901D1022100E0E2
:1051E00003216B780F221A40022A00D01146417029
:1051F00005204FE05420B080A888308168887081F5
:1052000028480078002801D1022000E003206A78B5
:105210000F211140022900D00846F071022C18D14C
:105220002148017831732149097871734178F181FE
:10523000807830821E48007870821E480088B082D4
:1052400062201D49085CF0821C48008830831A20C7
:1052500000E00C20009036180027194CE8198068EF
:105260002146FDF7D4FDFEF714F8F053F119000CB8
:1052700048803F1D402FF1D10098C019074E81B2E0
:10528000F82272547118F522CA70F6228A70F72239
:105290004A70001D80B201B0F0BDC046141300205A
:1052A000F4F3F2F1C80600201412002006130020C7
:1052B000241200208803002030100020CA0600209D
:1052C0000000C8422E090020F0B50A4801210170F3
:1052D00009494A88428002460832084BF0CBF0C2A6
:1052E000F0CBF0C2F0CBF0C2F0CBF0C20978417045
:1052F000F0BDC046EC070020D40F0020540F002062
:105300000F2801D8002070470120704700687047BF
:1053100010B586B0114802F0DEF801200390104964
:105320000A6802430A600968014000910220049063
:105330000C4802900820019000980520000701A960
:1053400000F05EFB0624204600F0DAFC0021204637
:105350000A4600F0E1FC06B010BDC046E00800209F
:10536000341002400000311007480821C160C160BC
:10537000C943064A13680B40136042680A40426002
:1053800002680A400260704700180240801802401C
:10539000014800787047C04634080020F0B585B059
:1053A000C16B03910E6801680F6804243A462240DD
:1053B000554255410490006CC6403246224053424B
:1053C00053412B432CD00291012202213B460B403A
:1053D0005D425D41B307144600D52C46049D20353F
:1053E000002C2DD0019008231F407C427C413307C4
:1053F00000D52246002A039C0498029940D10A68ED
:105400000E239A430A6001210A46019B9A4062607A
:10541000816300222A706970016B00292FD12FE06F
:105420000A68920603D40A6804239A430A601A4A57
:10543000134618339942049818D001239B0216E0B2
:105440000E4602990A68920605D40A680A239A430E
:105450000A6001226A7000222A700F4A134618332C
:10546000994204980ED001235B020CE04023151DE5
:10547000A94200D01C461460C16A002900D08847A8
:1054800005B0F0BD2023141DA14200D01E461660B9
:10549000816A0029F3D1F3E704000240F0B585B03A
:1054A00000282DD004460646203602207070A2CC7B
:1054B000236860680190A0680290E068039020690A
:1054C00004900868104A02402A433A431A4301985C
:1054D00002430298024303980243049802430A607D
:1054E0000025E56209482063357009480818142131
:1054F0000C3CFDF731FF800020640120707000E05B
:105500000125284605B0F0BD0FC0FFFF0000024096
:10551000F8FFFDBFF0B582B004462020255C0220D4
:10552000012D28D00192264620360122327077784C
:10553000012F1ED1022070700020A06326683768FA
:1055400097433760E56B0095276C1546BD40009F7B
:105550007D6073606368102B019F00D00F46B760B9
:10556000102B00D00199F160E16A002905D00E21CD
:1055700008E00021317002B0F0BD31680423994386
:1055800031600A2133680B43336031681143316065
:1055900002B0F0BDB0B5044600F0F6FA0546601C56
:1055A00002D004480068041900F0EEFA401BA04243
:1055B000FAD3B0BD30020020F0B587B00690A54AFE
:1055C0001078012802D1022007B0F0BD019101201E
:1055D00005901070A0480068C00A1C2101409F4837
:1055E00041589F4806680C68E7B29E4DA04BBE42EA
:1055F00029D1260C2E404268B24224D10269240AE5
:10560000E4B2A2421FD182684C68E6B2B2421AD11B
:10561000220C954C2240C468944214D142698C6893
:105620001C40A2420FD18269CC681C40A2420AD120
:10563000C2690C69A6B2B24205D1220C8B4C224041
:10564000046A944217D007604A882A4042604A7828
:1056500002610A798260CA88834C2240C2608A68EB
:105660001A404261CA681A4082610A8AC261498A44
:105670007E4A1140016206980068032818D002286B
:105680002AD0012800D0DEE07D20C40000F07CFAA2
:1056900006940419012005900604764D2F683740C2
:1056A0002ED000F071FAA042F8D3002F2DD0CAE01E
:1056B0007D20C40000F068FA0394041901200590CD
:1056C00007046C4D2E683E4039D000F05DFAA042D0
:1056D000F8D3002E37D0B6E07D20C40000F054FA95
:1056E00000940419012005900704624D2E683E4085
:1056F00060D000F049FAA042F8D3002E5ED0A2E0BC
:105700005D482860002F00D09DE000275148476089
:10571000686804210491084368600120C006574965
:10572000016000F031FA06994418286830427DD0B3
:1057300000F02AFAA042F8D30320059079E04E4801
:105740002860002E7FD100200290C043019908609C
:105750000698C36800690003C018834273D24248A8
:10576000401C696801436960FF200493186000F0E1
:105770000BFA039946182C683C4005D000F004FA57
:10578000B042F8D3032002E03B482860029805901D
:10579000049B0120C1026A688A436A60002C4DD1D3
:1057A00000031B180699C868096909030818834291
:1057B000D5D348E030482860002E44D10020029024
:1057C000C04301990860069842688068C00180184B
:1057D000824238D21F4802994160686802210391D1
:1057E00008436860FF200492106000F0CDF9009932
:1057F00046182C683C4005D000F0C6F9B042F8D3FA
:10580000032002E01C48286002980590049A03993E
:10581000686888436860002C13D1069948688968D5
:10582000C901081880328242D4D30CE0059712488F
:105830002860686804998843686004E00198036000
:1058400001E001980260002002490870059807B045
:10585000F0BDC046E812002004100240E8BA00087B
:1058600000210240FF010000FF070000FF3F000091
:10587000FFFF01001020024011800000214334127C
:105880000120C00703490A6802430A600868C04350
:10589000C00F7047142002400648C168002901D497
:1058A000002070470449016004490160C068C00FCE
:1058B0007047C0460820024023016745AB89EFCD01
:1058C000F0B589B00290002968D0A748029A8242B8
:1058D00001D0022200E00122052003070020029CE3
:1058E0009C42019000D00192064607460346009173
:1058F00025E0079D059EB540029C21682943216053
:105900001C210140079006988840D9088900611839
:105910000A6A824307980A62A168A943A160616884
:10592000089A91436160E168A943E16000995B1CBA
:105930000A46DA40001DB61C0837002A2ED0012284
:105940009A4015460D40F2D005960892182139402C
:105950000F2606968E4003241A460794A243834CD2
:10596000A2180392126E04963240019C8C40A2420F
:10597000BFD1039C60347E4A1168A943116051680D
:10598000A9435160794A1168A94311605168A9433C
:1059900051602168049A91432160AAE709B0F0BDE3
:1059A00080B5054800F020F904480178002901D1AC
:1059B0000121017080BDC046AC06002010130020FC
:1059C000B0B504460D4D2868204216D02C602C60DE
:1059D000062000F085F90820C04365490A680240A6
:1059E0000A60294608390A6802400A600C3D2968A5
:1059F000014029602046FFF7D3FFB0BD0C180240DC
:105A0000F0B589B00B68002B00D1AAE00E465649CC
:105A1000884201D0022200E0012205210907002767
:105A20008842009700D000923A4608973C46039679
:105A300011E029434D4A5160059A641C33681946A8
:105A4000E1403F1D08322546089CA41C08942C46C2
:105A5000002900D185E001252946A1400B40ECD06A
:105A6000029107940592069704937268074634469C
:105A700010261643122E0ED11C20069A10400F2617
:105A80008640079AD3089B00FB181A6AB24326691E
:105A9000864016431E62384603273A4608998A40D4
:105AA000036893436468264601973E408E401E4338
:105AB0000660D643122C14D8A5402E4A154210D0A9
:105AC00082683240039BDB68089DAB4013438360D0
:105AD000E206D20F079B9A40436802998B43134317
:105AE0004360C1683140039EB268089B9A400A43F4
:105AF000C260E100049D069F059A079C9DD5234640
:105B0000182414400F21A1401A46019B9A43174BB9
:105B10009A18136E8B430099A140194311661449DA
:105B200009687368DA0301D5294300E0A943079C9B
:105B30000F4A116051689A0301D5294300E0A94337
:105B40000B4A516009490968DA0201D5294300E08E
:105B5000A943064A116051689A0200D569E7A94332
:105B600068E709B0F0BDC0460004005000180240CC
:105B70008018024006000600002A02D01822815038
:105B800070472822815070471F4800687047C04600
:105B9000014800687047C046000EFF1FB0B50028DE
:105BA00017D0044600680E4901600E490160616823
:105BB0004160A1688160FFF7E7FF05462068C16882
:105BC000002908D0FFF7E0FF401B3028F6D903205A
:105BD000B0BD0120B0BD074901600020B0BDC04686
:105BE000CCCC00005555000000680249016000203F
:105BF0007047C046AAAA00001A48006802490A680D
:105C0000101808607047C0465C14002080B503205F
:105C100000F008F8002801D0012080BD00F055F800
:105C2000002080BDB0B505460E480168012400295A
:105C300016D07D20C000FDF78FFB01460A480068A2
:105C4000FDF78AFB01F0C6FA032D09D8002807D119
:105C50000024E0432946224600F05EF80348056030
:105C60002046B0BD30020020D000002034020020C9
:105C7000704780B501680A68920706D58A6892075E
:105C800003D502224A60FFF7F3FF80BDB0B50028BC
:105C900015D00446407B002804D100202073204604
:105CA00000F012F80220607307CCC368054D1D4058
:105CB0000D431543C560012060700020B0BD012078
:105CC000B0BDC046FFF1BFFF704710B511240121E0
:105CD0000022204600F020F8204600F011F810BD08
:105CE000002809D41F210840012181400348016098
:105CF000BFF34F8FBFF36F8F7047C04680E100E066
:105D0000002805D41F21084001218140014801607D
:105D10007047C04600E100E0002805D40322034696
:105D200093430A4A9A1803E00C220240064BD21809
:105D30008007C00E8901C9B28140FF2383401068EB
:105D4000984308431060704714ED00E000E400E061
:105D5000BFF34F8F034804490160BFF34F8F00BF6B
:105D6000FDE7C0460CED00E00400FA0510B56449FB
:105D70000A68064B134014C81A43224343688068DC
:105D8000134303430B60002010BDC046FFF1F0FF3A
:105D900010B5421E9041800301229203584B1C68AB
:105DA00094432018186008480368042213430360D2
:105DB000012901D130BF02E040BF20BF20BF0168F0
:105DC0009143016010BDC04610ED00E0F0B587B012
:105DD00081788907494F50D505900120049001072B
:105DE0003A46203A10680840039006D110680843EC
:105DF0001060106808400690069801920291404E8B
:105E00003068C00511D40498040230682043306023
:105E1000FFF7BAFE05463068204206D1FFF7B4FE10
:105E2000401B0228F7D9032542E0032528023968E0
:105E3000014013D0059A5269024091420ED0386851
:105E4000049909043A680A433A603A688A433A6016
:105E500001462C4A11403960C00742D13A682948AE
:105E6000024005984169114339600399002904D122
:105E7000019B1968029A914319600468E1071AD1DD
:105E8000A10722D4A10608D5012149023A46083AC1
:105E900013688B43C168194311600025A10507D51C
:105EA00003218A04083F3968914300690843386038
:105EB000284607B0F0BD394608390A6880239A435E
:105EC000436813430B60A107DCD5012109023A4660
:105ED000083A13688B43816819431160A106D3D433
:105EE000DBE7FFF751FE0646814C38688007B5D4E2
:105EF000FFF74AFE801BA042F7D9D9E75C100240A9
:105F000000700040FFFCFFFFF0B583B000284BD0CD
:105F10000D46029075480068012101910840A84291
:105F200014D2724908680126B04328430860704CB7
:105F3000FFF72AFE07466D4800683040A84205D0AA
:105F4000FFF722FEC01BA042F5D9BFE0029B1868F4
:105F50008107754C0DD5410704D507210903226837
:105F60000A4322600F21090222688A43996811437B
:105F70002160C0071BD127465C48006801263040DD
:105F8000A8422DD959490868B0430860584CFFF71A
:105F9000FBFD054655480068C00721D0FFF7F4FD1A
:105FA000401BA042F6D991E0012003B0F0BD5B6830
:105FB000042B6ED8990001A251588F46D15F00087A
:105FC000776000088560000893600008976000080B
:105FD0002146083909684905019860D403B0F0BD2D
:105FE000029A107840073B4606D50720000319683F
:105FF0008143D0680843186018688006400F06D0B7
:10600000186838210840082822D13A480FE018467D
:1060100008380168181F00680004400F042800D9E0
:1060200000208000354A10588904490FC84019687B
:1060300089093C220A40324989581F220A40D0402F
:10604000384908602F480068FFF7ECFD03B0F0BD49
:106050001868084010283CD15868C00744D1181F60
:1060600000680004400F042800D900208000234964
:1060700008584000DBE72146083909688903019880
:10608000ACD50CE021460839096889010198A5D5ED
:1060900005E0A16D00E0616D890701989ED521683A
:1060A0000722914319432160114FFFF76DFD06460A
:1060B00020683821014002984068C000814200D128
:1060C00059E7FFF761FD801BB842F1D9032003B007
:1060D000F0BD1A680A40F003202AA8D01A680A40C6
:1060E000182AA4D00020A2E70348A0E7002002401D
:1060F0008813000000366E01006CDC02C0B8000896
:10610000E0B8000834020020064800680649096823
:10611000890A1C220A40054989581F220A40D0409A
:106120007047C046D00000200810024020B9000887
:10613000F0B585B00127002800D128E2029703902E
:106140000078C0071FD103980078800748D40398CF
:106150000078000773D403980078400700D48FE1DB
:10616000F94A906838210140202900D0B9E0D06D6B
:10617000800700D480E10398C068002800D07BE14C
:106180000020012779E1F04CA06838220240114636
:10619000103948424841E168082A60D008405ED181
:1061A00003994868002808D08968002900D128E1AF
:1061B00022690C239A430A4322610521090488427B
:1061C00000D1FEE001210A04904200D1FFE0DF4A45
:1061D000521E2368134023608A0421689143F8E02B
:1061E000FC4CA668E0680127384038221640102190
:1061F0007140091848424841002E3BD0002839D14F
:106200002068BE02039A5169002900D1BFE007212E
:10621000C902884391690143216038022168014322
:106220002160FFF7B1FC05462068304200D0C0E095
:10623000FFF7AAFC401B0228F6D90327A7E1E54A8D
:10624000906838210140182933D1106E800782D51B
:106250000398006A002800D07DE7029F97E120683C
:10626000800300D46FE703984068002800D06AE7F5
:10627000029F8CE120684005039B03D558690028E4
:1062800000D184E101922246BC025068D24901400B
:10629000D86908435060FFF777FC0546CD48006891
:1062A00020425BD1FFF770FC401B0228F6D9032780
:1062B0006DE1106E0399096A002900D1A3E0012164
:1062C00008431066FFF760FC0546C248006E800771
:1062D00000D540E7FFF758FC401B03270228F4D9FC
:1062E00055E101263107D06B0840019006D1D06BF3
:1062F0000843D063D06B0840049004980091BD4FD0
:106300003868C0050FD43402386820433860FFF77E
:106310003BFC05463868204205D1FFF735FC401BA1
:106320000228F7D996E00398C768002FA94C0AD035
:1063300000698103890F00D17004032109042269D7
:106340008A4302432261052F6FD0012F71D0E06D87
:10635000B043E065E06D042188436CE0002E00D07E
:106360000EE10720C0029B4B1968814303988069A6
:106370000843186098688006400F00D1E8E09868EC
:10638000019A1040082800D004E19448EDE0390259
:1063900088432060FFF7F8FB05468E4800683042CE
:1063A00000D1D4E6FFF7F0FB401B03270228F4D905
:1063B000EDE06068884901400398C0690843606067
:1063C000C5E601218A042368134323600A04216877
:1063D00011432160002803D0C820FDF7FFF9B2E681
:1063E00001204404FFF7D0FB05467A4800682042AC
:1063F00000D1A8E6FFF7C8FB401B0327C828F4D943
:10640000C5E0029FC3E0012188431066FFF7BCFB93
:1064100005467048006E800700D49CE6FFF7B4FB89
:10642000401B03270228F4D9B1E0E06D04210143A9
:10643000E165E06D3043E0656F4EFFF7A5FB054673
:10644000002F0FD0E06D80070FD4FFF79DFB401B9E
:10645000B042F7D9002003270FE0FFF795FB401B60
:10646000B042F7D8E06D8007F7D40198002803D137
:10647000E06B00998843E0630120002800D186E0AA
:106480000398406A002810D0524B996838220A407D
:10649000102A0CD10128029F79D04E48C0680127EC
:1064A00038400399896A884271D100276FE0012240
:1064B00014061968A1431960560602280ED10292EB
:1064C000FFF762FB0546434B1868304217D0FFF7D1
:1064D0005BFB401B03270228F5D958E0D86890439E
:1064E000D860FFF751FB04463A4800683042DCD0E0
:1064F000FFF74AFB001B03270228F5D947E0039862
:10650000806A00280AD15968C90A1C220A403B49FE
:1065100089583B4A914201D2029F38E0D968029AD9
:1065200091430143D960186820431860FFF72CFBA2
:106530000446284800683042B7D1FFF725FB001B0E
:1065400003270228F5D922E0001002400000FFFFD7
:10655000196858680004400F042800D90020800002
:10656000204A10588904490FC840996889093C227B
:106570000A401D4989581F220A40D0401B49086023
:106580001B480068FFF74EFB002800D1DFE5F8B29A
:1065900005B0F0BD9868104010280DD1D868C0072C
:1065A00016D158680004400F042800D9002080004C
:1065B0000C4908584000D8E7996811400120C003F1
:1065C0002029D2D0996811401829CED00020CCE7DC
:1065D0000348CAE7001002400000FFFF00366E01CA
:1065E000006CDC02C0B80008E0B80008D000002051
:1065F00034020020007000408813000040B90008F9
:106600000024F4000248016802220A430260704735
:1066100010E000E0B0B5002811D00446054648352A
:106620000220687020680168402291430160204682
:1066300000F05CF80020E06428706870B0BD0120B4
:10664000B0BD000080B5C16C01A004F093FD80BD19
:10665000687370692D3E4572726F72436F64652076
:106660003D20256420000000F0B581B0002838D01E
:106670000446054648356878002804D10020287073
:10668000204600F057F80220687021680868402210
:106690009043086001225002A36918406668A76809
:1066A000374326693E43676937430743E069384308
:1066B000266A06430E60E6680B4F0020BE42009239
:1066C000174600D307463F031B0C04221A40BA1892
:1066D000636A134333434B60E0640099697001B00F
:1066E000F0BD012001B0F0BD01070000B0B50068A9
:1066F0005B49884200D0B0BD012420030C490A68E0
:1067000002430A600A6882430A60052005072021C7
:106710002846FFF7D5F840212846FFF7D1F8802119
:106720002846FFF7CDF850482146FFF7C9F8B0BD1D
:1067300030100240F0B58BB0026849498A4201D05E
:106740000BB0F0BD0390474B186801252843186033
:10675000186828400690069818682843186018683A
:106760002840069006981868284318601868284042
:1067700006900698196802200143196019680140C3
:10678000069106992903DA680A43DA60DA680A4052
:106790000692069900260A960890079020200190FC
:1067A00006900320029009900520040706AF2046BA
:1067B0003946FFF725F90A964020069020463946CB
:1067C000FFF71EF90A968020009006902046394671
:1067D000FFF716F90A96069523483946FFF710F990
:1067E0002049486828434860486828400590059833
:1067F000C8682843C8601D4F1D4C50C704963E60B2
:1068000000987860C868039E284005900598680342
:1068100001993961786107200002F168083F8142DF
:10682000284600D804980102800239617861384610
:10683000FEF734FE029800032168814321607764EB
:106840007E622168014321600A24204604992A4679
:10685000FFF762FA2046FFF753FA0BB0F0BDC046CF
:106860000030014034100240000400506406002053
:106870001C000240F0B587B017460E460446412082
:106880008100254648356068884203D1A068002809
:1068900000D1A8E02878012802D1022007B0F0BD7D
:1068A00003A88AC001272F70FFF76EF90690687859
:1068B000012800D094E0002E38463A46059F00D1CA
:1068C000B4E0002F104600D1B0E0029220680168C9
:1068D0004022019291430160042169700023E36426
:1068E000E786E385A7862663A385A362A363E363A4
:1068F00007210902E268012605918A42374600D93C
:106900001F463B0337034168B943C9184160F1038F
:10691000A3688B4204D10121890303688B43036080
:1069200001684906049E039F03D40168019B194333
:106930000160E08E0599491C8A420AD322E0007B5F
:10694000216B0870206B401C2063E08E401EE086A7
:10695000E08E002827D020688168C907EFD1FFF7B3
:1069600013F9711CF4D00699401AB042F0D30320F9
:106970005BE0216BC0680880881C2063E08E401EAD
:10698000E086E08E00280ED020688168C907F0D12B
:10699000FFF7FAF8711C03D00699401AB042E6D20C
:1069A000E08E0028F0D16068B8420CD1A0680121C7
:1069B000CA03904202D08902884204D1206801684B
:1069C000019A9143016020463146069A02F016F979
:1069D000002813D0E06C20210843E064E16421E04A
:1069E00002203A4622E00420687000932046314697
:1069F00032463B4600F0E4F907B0F0BD6068B842AB
:106A000010D1A0680121CA03904202D089028842B5
:106A100008D10320410220463246069B02F086F848
:106A20000028D7D1E06C411E8841029A00212970CC
:106A30006A7007B0F0BD0000F0B583B013460A4697
:106A4000054680682E46483600280CD14121890031
:106A50006C688C4207D1042070702846114600F003
:106A6000C5FA04467DE03178012901D1022478E09D
:106A700001243470717801292CD1002A6FD0002BA9
:106A80006DD029680C6840270197BC430C60042432
:106A900074700024EC64EB86AB862A63AC63EC6311
:106AA000AC85EC8501230293DB03984204D10120DD
:106AB00080030B6883430B6048682B4B1840486089
:106AC0004B68E868BD4FB84206D3012000038343FA
:106AD0004B601FE0022442E0029F380303434B60F7
:106AE000BB026F6C7F699F4214D14B6883434B603C
:106AF000EB8E4868DB0705D11B4B18404860E88ED9
:106B0000400806E0029B5B0318434860E88E40089B
:106B1000401CE886686C164F164B8362134BC362A9
:106B200007634463EB8E0C31FEF7F4FC002806D0BB
:106B3000E86C10210143E964029C74700FE028683E
:106B40000168490603D40168019A11430160416854
:106B500020220A434260416801220A434260002029
:106B60003070204603B0F0BDFFDFFFFF4D88000806
:106B70002B8800086188000870B52748016820222A
:106B80000A4302602548012444700F4D6888244E52
:106B9000301881780A0943781B071B0ED218490167
:106BA00023020B40D1181F4AD28A00F003FF0128AC
:106BB00009D16888305CAA2805D102F015FA02F0E4
:106BC00025FA1948047070BDE0070020B0B51248DE
:106BD000016840220A43026010480125057028021E
:106BE0000F4CA1784A010240080961780907090E93
:106BF000401881180B48C28A204600F0DBFE0128AD
:106C000008D12078AA2805D102F0EEF902F0FEF9A9
:106C100005480570B0BDC04604000240B811002010
:106C2000A8100020D40F00202A100020F0B589B051
:106C3000079304464820205C012801D10226B9E0D0
:106C4000154606912646483601273770FEF79CFF09
:106C500033467178012941D10590069800283E46B7
:106C600000D1A4E0002D3E4600D1A0E004972068AA
:106C70000268402102918A430260032603935E70FA
:106C80000021E164E585A585069FA762A1862163B1
:106C9000A163E1630191E1860122D303A1689942D6
:106CA00003D1910302680A4302600168490603D4D4
:106CB0000168029A1143016061684A424A416B1EB1
:106CC000594259411143E268C74B9A4208D30029FF
:106CD000079D0ED03988C160B81C06E0022666E028
:106CE0000029079D21D0397818E0A062E08D401E70
:106CF000E085E08D00282BD020688168890708D4C2
:106D0000FEF742FF691CF4D00599401AA842F0D35F
:106D10004BE0A16A0A88C260881CE6E70173A06A9A
:106D2000401CA062E08D401EE085E08D00280FD061
:106D300020688168890708D4FEF726FF691CF4D013
:106D40000599401AA842F0D32FE0A16A0978E5E737
:106D50002E460325E90220463246059F3B4601F0B8
:106D6000E5FE00280ED1204631463A4601F046FFA6
:106D7000002807D16902204632463B4601F0D6FE84
:106D8000002804D0E06C20210843E064E164A0689E
:106D9000002807D1019808902068C1680891806890
:106DA00008900898E66C701E8641049F039B0020A3
:106DB00018705F70304609B0F0BDC0460107000092
:106DC000F0B587B004464820205C012802D102209B
:106DD00007B0F0BD1D4604920591274648370126AD
:106DE0003E70FEF7D1FE324606467978012900D082
:106DF00083E005980028104600D1EEE004980028B2
:106E0000104600D1E9E0002D104600D1E5E00392E4
:106E10007878042801D005207870019720680168EF
:106E200040220092914301600022E264E586E585FC
:106E3000E168DD4F01230291B942194600D31146A2
:106E4000069609031B0347689F437918416004991C
:106E50002163A586059FA762A263E263A5850168F9
:106E6000490603D40168009A114301600C9E6168D1
:106E70004B424B41691E4A424A411A430299CA4B4E
:106E8000994248D3002A06D03988C160B81CA06254
:106E9000E08D401EE0850125019FE08D002802D194
:106EA000E08E002877D02068816889070DD5E18DB4
:106EB00000290AD0012D08D1A16A0A88C260891C64
:106EC000A162E18D491EE18500258168C9070BD0CB
:106ED000E18E002908D0216BC0680880881C2063DF
:106EE000E08E401EE0860125FEF74EFE711CD4D0D8
:106EF0000699401AB042D0D34BE003924120820061
:106F000063680220934267D1A268002A64D10429F1
:106F1000039A62D16DE7002A07D039780173A06A1D
:106F2000401CA062E08D401EE0850125019FE08DA0
:106F3000002802D1E08E00282DD0206881688907C2
:106F40000ED5E18D00290BD0012D09D1A16A097858
:106F50000173A06A401CA062E08D401EE085002500
:106F600020688168C9070CD0E18E002909D0007B18
:106F7000216B0870206B401C2063E08E401EE08671
:106F80000125FEF701FE711CD1D00699401AB042CE
:106F9000CDD3032020E003200590C10220463246D5
:106FA000069D2B4601F0C2FD00280FD12046314638
:106FB0002A4601F023FE002808D105984102204608
:106FC00032462B4601F0B2FD00280BD0E06C2021A8
:106FD0000843E064E1640120039A002139707A706B
:106FE00007B0F0BD0020F7E701070000F0B585B05D
:106FF00004464820205C012802D1022005B0F0BDE3
:107000002546483501262E706F78012F30D1002992
:1070100055D0002A55D0002B304600D1C0E00E4696
:1070200003926878042801D00520687004952168CF
:10703000086840220292904308600022E264E385DF
:10704000E386032040034D6885434D60A385A66217
:10705000A38603982063A263E2634E68E068524D02
:10706000A84217D30120000386434E60049D4AE0E6
:10707000039104954125A900656802208D4200D046
:107080008DE0A568002D00D089E0042F049D0399B0
:10709000BDD085E00120050301952E434E600746D3
:1070A0008602206C4069B042049D13D14868DB071A
:1070B00009D1BB0398434860E08D400809E03046A1
:1070C0006EE030466CE0BB0318434860E08D40083A
:1070D000401CE085606C4069B04214D14868019B57
:1070E00098434860E38E4868DB0705D17B039843EB
:1070F0004860E08E400805E07B0318434860E08E5E
:107100004008401CE086606C284B036342636B7848
:10711000042B01D0274E00E0254EC6621546042BF5
:1071200001D0264B00E0244B8362E38E0C31039A9E
:10713000FEF7F0F9002807D0E06C10210143E1646C
:107140000120049D68702BE02268506801263043BE
:107150005060206C8562C56205634563E38DA16A5A
:107160000C32FEF7D7F9002807D0E06C102101435C
:10717000E164049D6E70304612E02B462068016881
:10718000490603D40168029A114301604168202234
:107190000A434260416802220A4342601846049D45
:1071A0000021297005B0F0BD010700002B88000800
:1071B0004D88000857880008618800081F8900086A
:1071C0007047704702490A6802430A607047C04628
:1071D0001C000140401E010E01D0012070470749EC
:1071E0000B4A5060064803680B4003218907591871
:1071F000016000209060072111607047FFFFFF00D1
:1072000020ED00E0024801680222914301607047CE
:1072100010E000E070477047B0B5002819D0044670
:1072200005463C356878002804D1002028702046A7
:1072300000F04EF802206870206803681F498842F9
:1072400002D01F4A904206D170229343A2681A438B
:1072500002E00120B0BD1A461A4B984208DD884270
:107260000CD0194B984209D0184B984206D022E016
:10727000134B984202D0944B98421CD103231B021B
:107280009A432369134380229343A2691A430260FD
:10729000E268C26262688262884205D00A49884216
:1072A00002D00A49884201D161690163012141612B
:1072B00069700020B0BD1346E5E7C046002C0140D0
:1072C00000040040FF2B0140004801400044014001
:1072D00081B00120C00305490A6802430A600968B9
:1072E00001400091009801B07047C0464010024034
:1072F0000068C26801210A43C26082680723134004
:10730000062B02D002680A430260002070477047D3
:10731000B0B504468020C54320680169890716D5A9
:10732000C168890713D529467E3101610121217782
:107330008069800703D02046FFF7E9FF05E020467B
:1073400000F08AF8204600F088F8002020772068B6
:107350000169490717D5C168490714D529467C3109
:1073600001610221217780698005800F03D02046CA
:10737000FFF7CDFF05E0204600F06EF8204600F054
:107380006CF80020207720680169090716D5C168CC
:10739000090713D529467831016104212177C06995
:1073A000800703D02046FFF7B2FF05E0204600F03B
:1073B00053F8204600F051F800202077206801693A
:1073C000C90617D5C168C90614D5294670310161AF
:1073D00008212177C0698005800F03D02046FFF780
:1073E00096FF05E0204600F037F8204600F035F81B
:1073F0000020207720680169C90708D0C168C90743
:1074000005D029467F310161204600F027F8206829
:107410000169090606D5C168090603D5056120463C
:10742000FFF7F8FE20680169490608D5C1684906DA
:1074300005D5294640310161204600F04BF820680F
:107440000169890607D5C168890604D560350561DB
:107450002046FFF7E0FEB0BD7047704780B5194881
:1074600000681948016801229143016003F0CCFAD9
:1074700003F0C4FA01F0D2FD6420FCF7AFF901F08B
:10748000BBFD02F067FA032000F090F9192080019B
:10749000FCF7A4F90020FEF7C5FBFDF779FF0328F0
:1074A00002D101F013F804E008480078012101F04E
:1074B000B9F801F051F8064840884004000C01F08A
:1074C00079FA80BD0444004000200040D40F002021
:1074D000E00700207047B0B5002813D004460546E9
:1074E000443524206870012040032168CA68824323
:1074F000CA60204600F06AF80020A0646870287016
:10750000A870B0BD0120B0BD0C4901600A490868EF
:1075100000220A607047C04606490968890607D5F7
:107520000068406804490A68044B9854501C08607D
:107530007047C0460044004050140020D013002083
:10754000F0B581B000283DD0044605464435687842
:10755000002804D100202870204600F04FF8242095
:10756000687001277E032068C168B143C16020466E
:1075700002F01CFA2021605C400611D53A03206815
:10758000436993430096666A334343619642009E83
:1075900006D10322520343699343A26A1A4342610C
:1075A000F8022268136983431361506908239843E2
:1075B0005061D0683043D0600020A0646970A97029
:1075C00001B0F0BD012001B0F0BD000010B50120F8
:1075D000400409490A6802430A600A6882430A6053
:1075E0000520040704212046FEF76AF908212046F9
:1075F000FEF766F910BDC0462C100240F0B583B00E
:10760000184801680124214301600168214002916A
:107610000299610482680A438260134D04270222A2
:1076200012232F606B60AC60EA602F6180680840B5
:10763000019001980520060730462946FEF7E0F93B
:107640002F610820286030462946FEF7D9F91C250D
:10765000002128462246FEF75FFB2846FEF750FB36
:1076600003B0F0BD3410024050060020F0B585B0E4
:107670000F4604460546443568780221202816D175
:107680000120002F00D18BE01646002A00D187E0B0
:10769000012001900203A068009290420AD1F807ED
:1076A00008D02069002805D1019805B0F0BD084632
:1076B00005B0F0BD28780128084671D00493002059
:1076C0000390A0640198287021206870FEF75CFA8E
:1076D000029066862686A0680099884202D12069B9
:1076E000002801D03E4601E000260397049A08E0F6
:1076F000002E12D0307821684860761C608E401EC3
:107700006086608E002820D0206800680006EFD4D4
:10771000571C18D0002A0FD120E0039B188821495C
:107720000840216848609B1C03930026E6E7016837
:107730000906DDD4002FFAD0FEF726FA049A029942
:10774000401A90420AD82068F1E720680068400695
:1077500021D4002A02D0561C0FD014E00D20400185
:107760002168CA688243CA604869019A90434861A7
:1077700020206870A870032010E020680168490686
:1077800009D4002EFAD0FEF7FFF90299401A0499A5
:107790008842F2D9E2E72020687000200021297099
:1077A00005B0F0BDFF0100007047000080B582B059
:1077B00005480168406801900091684600F0F4FEB9
:1077C00001F024F902B080BDD8B80008B0B582B08D
:1077D000144601AD0020A87068708020084328700E
:1077E0000A4803220A4B2946FFF744F8002803D031
:1077F00008A004F019F8FEE701A88178407800029B
:1078000040182080002002B0B0BDC046C01100204A
:1078100088130000505933325F5350495F526561FD
:10782000645F52656773204572726F720D000000CD
:1078300010B582B001ACA2702170100A60700748C8
:107840000322074B2146FFF7F1F9002803D005A0DA
:1078500003F0EAFFFEE7002002B010BDC0110020D7
:1078600088130000505933325F5350495F57726993
:1078700074655F52656773204572726F720D000008
:10788000B0B5FBF7D7FF401C04D023481E21FBF7FF
:10789000C7FF38E0204C2046163020A110252A468C
:1078A000FBF738FA2046563020490C22FBF732FA13
:1078B000204646301EA12A46FBF72CFA20463630D9
:1078C0001BA12A46FBF726FA204626301CA12A4691
:1078D000FBF720FA62201E4921521E481E496166AC
:1078E000A066E066206760670A201C491C4A1D4BA1
:1078F0000BC42260616001200003208178210C3CD0
:107900002046FBF79BFF00242046214600F08AFE1C
:10791000204601F051FBB0BD301000204040292529
:1079200023232121212121212121212130BB0008D4
:1079300040402927232321212121212121212121E7
:1079400040402923232321212121212121212121DB
:10795000140900001E1E1E1E040078000001010014
:107960000100001000102200F0B581B01E4617463D
:107970000C46009018461146FBF741FA0546204692
:107980002146FBF7EBF93946FBF739FA3146FBF7AD
:1079900036FA0146FBF7E2F901462846FBF774FA8E
:1079A00004460098FBF755FC01462046FBF7D6F944
:1079B00001B0F0BDF0B581B006460D4F3878884271
:1079C0000FD114460D46401C1146FBF7C5FC39701B
:1079D000E9B2304603F070F9E843011948424841E2
:1079E00002E000203870FF2040B201B0F0BDC04678
:1079F000A8060020014800787047C046300C0020DF
:107A000080B50248FEF735F980BDC046B8060020B3
:107A1000F0B595B0524F388800282AD151480168F6
:107A200011914168129181681391C16814910169A3
:107A3000109141690F9181690E91808B0D904A4898
:107A4000F0C81038034610330ECB808B0891099292
:107A50000A930B90109800900F9801900E98029046
:107A60000D9803A9F1C13E4F11AB0FCB00F0FDF80B
:107A700038803E4C80212046FBF765F93C48402584
:107A80002946FBF760F93B482946FBF75CF93A7851
:107A90003948032110252B4603F014F832480078AA
:107AA0000F211491084002281FD13A780095324DD9
:107AB00001210023284602F0ABFF304E3078401CF5
:107AC00030702948808A00F085FEFBF7C9FB01462B
:107AD0003078FBF741FC3170002906D10C3528487D
:107AE00010221823294601F06DFA3888002801D0A9
:107AF000002038800025234E70598012FBF79EFB32
:107B000060516719701940688012FBF797FB786025
:107B10000835802DF0D1154C15491022204602F071
:107B20004DF91148007814990840022815D1002514
:107B3000154E70598012FBF781FB6051671970195F
:107B400040688012FBF77AFB78600835802DF0D111
:107B500006480E49102202F031F915B0F0BDC046BA
:107B6000D4000020F40F0020D40F0020BC0D002012
:107B7000540F00207C0E0020080600201312002065
:107B80008C03002030090020B00900203C0E0020AA
:107B9000F0B583B005290ED20022002907D00B468C
:107BA0000488121992B25B1E801C002BF8D110467B
:107BB000FBF7D2FB55E04A1E0292012A1EDB00248D
:107BC0002246019105E0521CD4B20299A1420199CA
:107BD00014DDE3435C18012CF5DB0026354603E099
:107BE0006D1CEEB2B442EEDD7300C65AC7187B8836
:107BF0009E42F5D9B91C3B800E80F1E7092901D3DB
:107C0000022400E001246200CB0713D1E4434B08B7
:107C10001B19911C00252A462C465D196D00455BF9
:107C2000521992B2641CE5B2A942F6D81046FBF78D
:107C300093FB16E001210A43029BD90F5918491002
:107C40000B1B002529462C465D196D00455B491923
:107C500089B2641CE5B2AA42F6D808461146FBF781
:107C60007BFB80B203B0F0BD7047B0B50546089805
:107C7000C4B22046FDF744FB0146002000290FD185
:107C8000E9B2A1420CD005990D9A01208A4207D190
:107C900006990E9A4A40D1B2002901D16042604152
:107CA000B0BD000070B586B01F48016820221143A6
:107CB00001600068104000900220049000240394AA
:107CC00001200290082501950098064E01A9304632
:107CD000FDF796FE304629462246FDF74DFF06B0D9
:107CE00070BDC0460014005070B586B001200290EF
:107CF0000D490A6802430A600968014000910221A7
:107D000004910024039405030195009805200607BB
:107D100001A93046FDF774FE304629462246FDF79C
:107D20002BFF06B070BDC0463410024070B586B05F
:107D3000044600260596400603D0FF2670B206B022
:107D400070BD0D46FDF7A8FD02950194022000903C
:107D5000684605A9FDF730FC002800D0FEE7FDF7D6
:107D60008FFDEBE770B50D460646FF20B1070FD13A
:107D7000144691008919074A914209D8FDF78CFDF4
:107D8000304629462246FCF757FDFDF779FD0020D5
:107D900040B270BD00000108F0B58BB000200A9021
:107DA00009900890E64D802628463146FAF7CBFF29
:107DB000E4483146FAF7C7FFE34840263146FAF770
:107DC000C2FFE2483146FAF7BEFFE148008880076B
:107DD00006D1E0490C31E0481022182301F0F2F8F6
:107DE000DE4C2278DB4F032110263846334602F062
:107DF00069FE22780096012100263846334602F0BB
:107E000007FE2088002800D02680D54CA05980127B
:107E1000FBF714FACB490F468851D248805980129B
:107E2000FBF70CFAA851BF19A01940688012FBF7A4
:107E300005FA7860AF19CB48801940688012FBF7CB
:107E4000FDF978600836802EE0D1BE48BF49102584
:107E50002A4601F0B3FFBA4CBB49204607952A4693
:107E600001F0ACFFBA48008804281AD30026BE4FA0
:107E700002E0361D402E14D0F8488559FB48815940
:107E80002846FBF769F9002801D1F8488551F248E6
:107E90008559B9592846FBF75FF90028E9D1BD514A
:107EA000E7E7F34E327807980090EE48032100256B
:107EB0002B4602F057FE3088002800D03580ED4E6A
:107EC00070598012FBF7BAF9605167197019406850
:107ED0008012FBF7B3F978600835802DF0D1DF4EC2
:107EE000402530462946FAF72EFFDA4C102220466C
:107EF0003146019201F062FFDF48032231460492CD
:107F00002B4601F05FF8DD480178032901D2491CB6
:107F10000170007802F082FED1480088082800D263
:107F20009AE007900027D64E02E03F1D402F09D06F
:107F3000CA48C559F1592846FBF70EF90028F4D173
:107F4000F551F2E70798082800D285E03ED1C14CF0
:107F5000002705E0CE48C6513F1D0834402F7BD096
:107F6000C0480546C05FFBF769F92060E8190221A7
:107F7000405EFBF763F9606001222046C14D29464F
:107F800001F01CFF2868FBF7B7F9BF4ABF4BFAF7AF
:107F9000B9FF06460D46B148C059FBF7ADF9BA4ADC
:107FA000BA4BFAF7AFFF02460B4630462946FBF7BD
:107FB0005BF8FBF7B5F90646FBF79EF9B54AB64BF9
:107FC000FBF726F90028C5D1B44EC3E7002703E02C
:107FD0003F1D0834402F3FD0A2480546C05FFBF745
:107FE0002DF92060E8190221405EFBF727F9606057
:107FF00001222046A34D294601F0E0FE2868FBF748
:108000007BF9A14AA14BFAF77DFF05460E4693483E
:10801000C059FBF771F99C4A9C4BFAF773FF024673
:108020000B4628463146FBF71FF8FBF779F9054662
:108030009748C0592946FBF78FF806462846FBF7B4
:108040005BF9002EC4D1934A934BFBF7CBF8002881
:10805000BED18F48C551BBE781480088800700D05A
:10806000F6E08F4800780F2802D8401C8C49087031
:108070007D4C8C4E8C4F06E0059C241D5B1C0493AC
:10808000092B00D1E4E040213046FAF75CFE35468A
:10809000182638463146FAF756FE8148027801988C
:1080A000801AC1B20F2905940291039224D84E433D
:1080B00088002D184C1C0027079706970599885FA4
:1080C0002880891902228F5E6F80FBF7B7F801467E
:1080D0000798FAF743FE07903846FBF7AFF80146DA
:1080E0000698FAF73BFE0746601C18362D1DE1B2D4
:1080F00010290446E1D101E000270797079A039869
:10810000102833D10024674E0792305F0001FBF73F
:1081100095F80799FAF773FEFBF7A2F83053351973
:108120000220285E0001FBF789F83946FAF767FE5E
:10813000FBF796F86880241D402CE6D150E0C0463D
:10814000BC0D0020D40E00203C0E0020540F002057
:108150002E090020080600208C030020D4000020F7
:1081600030090020B0090020CC06002002990F2918
:108170004C4E35D81446FBF76CF80646204631467F
:10818000FAF782FE079038463146FAF77DFE05463B
:10819000029A900043490F18541C0220385EFBF7E6
:1081A0004DF82946FAF72BFE8321CE053146FAF722
:1081B0002EFEFBF755F87880388800B2FBF73EF8C2
:1081C0000799FAF71CFE3146364EFAF720FEFBF708
:1081D00047F83880601C3F1DE1B210290446DCD10D
:1081E000002401253148314622462B4601F082FC0D
:1081F00030460A302C4F395BEA43825E5243120A02
:108200008918028812B25243120A89183953001D84
:10821000A41C182CEFD126480A902648099026481D
:10822000089008A900220B23384602F01CFEB9482A
:1082300000880728049B00D81EE758001F494018F3
:10824000801F0288F98A8A4200D315E7018013E76C
:108250000BB0F0BDBC0D00203C0E0020540F0020E0
:108260002E090020080600208C030020480300206F
:10827000D6000020300A00202812002029100020FB
:108280000C070020C01300202D431CEBE2361A3FE0
:10829000940F002048E17A14AE470940CDCCFC4150
:1082A0002B1000207C0E0020BC0E002020BB0008FC
:1082B00008090A0B04050607000102031812002032
:1082C000F0B587B003910590AA4A10780F210140BC
:1082D000012903D0508B401CC5B200E01025147F4B
:1082E000FF27A54200D89CE00097681E0190274612
:1082F00002950BE01046FAF73DFF002800D190E010
:108300007F1CFCB2A5429B4A00D889E0A1000598D9
:1083100004914058958BF9B28D4206901CD1FAF722
:10832000EBFF414A414BFAF7EDFDFAF7F9FF03F095
:10833000A9F93F49FAF76BFD06460398005DFAF785
:1083400088FF01463046002D45D0FAF713FF00287C
:10835000029D069ED4D155E0FAF7CEFF324A334B48
:10836000FAF7D0FDFAF7DCFF03F08CF93049FAF7A1
:108370004EFD06460198A04210D1029D102D35D326
:108380000398C07BFAF765FF01463046FAF7F2FE24
:108390000028069AB4D10598816BABE70398005D7D
:1083A000FAF757FF01463046FAF7E4FE0028029D2F
:1083B000069EA5D1059804990C18201F0168304627
:1083C000FAF7D8FE00289BD161683046FAF7E0FE44
:1083D000002895D025E0FAF7CDFE0028029D069AE8
:1083E0008ED1059804990818416883E70398005DC9
:1083F000FAF72FFF01463046FAF7BCFE0028069E2A
:1084000000D07DE7059804990C18201F01683046BC
:10841000FAF7B0FE002800D072E7616830466AE7DC
:10842000009FF8B207B0F0BDFCA9F1D24D62503FF9
:108430000000A0417047000010B582B0FDF7E6FBD8
:10844000FBF77CF91A48002107225202194B0360FE
:1084500042608160FDF71AFC002800D0FEE7012091
:10846000000715490A6802430A6009680140019142
:108470000198FDF7CBFB1148FDF78CF801F0F4F9FA
:1084800000F09EF801F066FA03242046FFF78EF90B
:108490000B480C490C4A14C001600838FDF77EFBFC
:1084A000002800D0FEE70648FDF79EFB02B010BD95
:1084B000B8060020007C00403C100240B80B0000D1
:1084C000AC060020102700000030004010B5104816
:1084D0008021FAF738FCB948002101700D4801806D
:1084E000AF48012404800C480170AE48048003208A
:1084F000C1010A48FAF727FCA648C4822103018378
:1085000035218182FCF726F902F020FE10BDC0461D
:10851000BC0D00202E0900202B1000208C03002011
:10852000F0B581B000240A4D144E0A4F02E0641CDD
:10853000022C0BD0285D0028F9D0728820465043C9
:1085400080B23918E0B2FCF765FBF0E701B0F0BD8E
:10855000B8110020A81000208E48417E890090228A
:10856000054B9952C28A054B9A80007E18700831DB
:1085700059807047D40F00204C070020E0070020EE
:10858000054800687047C046002904D0024A08CA5E
:1085900008C0491EFBD1704780FB000801490860F4
:1085A0007047C046B80D00204168034A116000685A
:1085B000024908607047C0460C13002008130020D1
:1085C00070B586B0012002900D490A6802430A6026
:1085D00009680140009102200490002403941025B2
:1085E000019500980520060701A93046FDF708FA15
:1085F000304629462246FDF7BFFA06B070BDC04698
:108600003410024080B50520000710210022FDF73C
:10861000B3FA80BD80B50520000710210122FDF7C7
:10862000ABFA80BDF0B589B00C4601AA0021918358
:1086300007910691059104910391029101911028EF
:1086400003D201A8FF22428021E012280FD0112876
:1086500019D101A9FF204880112008704C48828957
:10866000CA8242898A8201460F310E3016E001A883
:10867000FF214180122101704548016906910146A0
:10868000153114300AE001A8FF214180102101704A
:108690003F4841680691014609310830007801AB36
:1086A00018760878587663213948425C19780907AA
:1086B00001D0114609E06421415C89180F2903D8D3
:1086C000022A02D8511C00E00F2101AD6983652107
:1086D000405CA883284602F0EBFC2E4829464CC992
:1086E0004CC0CCC9CCC00988018008480ECD0EC052
:1086F0004ECD4EC02988018000F00AF8002C03D02E
:10870000FCF728F802F022FD09B0F0BDF40F0020BC
:10871000B0B51E480025058062201D490C5C1D482F
:10872000808A00F057F80146204602F0FBFC1A4907
:1087300008801A4805701A480121018019480180F3
:1087400019480570194805701948057019480570D1
:1087500019480560194805701948057045708570FD
:108760001848057045708570C570057145711648CB
:108770004021FAF7E8FA1548056045608560C56054
:10878000056113484821FAF7DEFAB0BD88030020DE
:1087900030100020D40F0020CA0600209A130020B9
:1087A000D4000020D60000202C1000202A10002029
:1087B000C806002013120020C0130020291000203A
:1087C0001412002094130020540F002014100020D5
:1087D000EC07002080B50021124A1388834204D0A0
:1087E000921C491C1029F8D11021481CFAF726FDCB
:1087F0003F210906FAF70BFB80BDC04680B5FAF7AA
:108800007BFD0022064BFAF77DFB02460B46FAF78A
:1088100079FBFAF753FDC0B240000249085A80BD07
:108820000000E0BFD8000020704780B5406A0168B2
:108830004A6803239A434A60C16C10220A43C26407
:10884000492101224254FDF7FDFE80BD80B5406AFA
:10885000FEF7BCF980BD80B5406AFEF7B2FC80BD72
:10886000F0B581B00646446AFDF78EF905463068DA
:10887000006880064ED4206841682026B1434160DC
:10888000A1684122970003220092D243002902D11D
:108890006368BB4200D0921C436813404360626827
:1088A000BA420AD10122D303994202D092029142E4
:1088B00003D10168402291430160642120462A4689
:1088C00000F09CF9002804D0E06C3043E064E664DA
:1088D00013E06068B84210D1A0680121CA03904239
:1088E00002D08902884208D10098410264222046C1
:1088F0002B4600F01BF90028E6D10020E086492035
:1089000001212154E06C002804D02046FDF79AFE96
:1089100001B0F0BD2046FEF72FF901B0F0BDF0B573
:1089200081B00646446AFDF72FF9054630680068B5
:10893000800634D4206841682027B943416003266B
:10894000F102642220462B4600F0F0F800280ED1F8
:10895000642120462A4600F051F9002807D171020F
:10896000642220462B4600F0E1F8002805D0E06C98
:108970003843E064E06C3843E06420684168B14308
:1089800041600020E085E086492001212154E06C0F
:10899000002804D02046FDF755FE01B0F0BD20466A
:1089A000FEF70EFC01B0F0BD80B51448FDF732FEB5
:1089B00080BDC04610B511480821114A0023072484
:1089C00024020CC0036044608360C36003614161A2
:1089D0000124E1038361C1610838FDF745FE0028E9
:1089E00000D0FEE76002FEF7EDFB06484088400439
:1089F000020C02480449FEF71FF810BD3808002099
:108A000000300140E0070020A8100020F0B58DB034
:108A1000424D00262E6218210124A20407231802C9
:108A200041239F003E4B88C52E6005906860AE6074
:108A3000EE602A6169614921083D685C0028069161
:108A400040D14820049400242C540C940B940A9494
:108A50000994089401239903324882680A4382608A
:108A600082680A400792079901681943016001680A
:108A7000194007910799016802220292114301608F
:108A8000006810400790079803930C93032001900F
:108A90000B900A93099204200890234808A900919A
:108AA000FCF7AEFF0C94049C01980B9003980A907D
:108AB0000298099005980890052000070099FCF796
:108AC0009FFF06990220685428680168402291435C
:108AD0000160FC37A9690F406A68AB6813432A69D3
:108AE0001A436B6913433B43EA691A432B6A1343E6
:108AF0000360EA68059B9A422346274600D933461D
:108B00001B03090C04240C4019196B6A0B43134313
:108B10004360EE6406982F540DB0F0BDC0110020E4
:108B2000003800403410024000040050F0B589B015
:108B30001F4614460E46029007A800250570FDF753
:108B400023F8381A06940419FDF71EF8029A0490C7
:108B50005248006823214143080D05946043089062
:108B6000106803908068304228D010464830019049
:108B700004E025461068806830421DD00327780243
:108B8000864204D10398007B07A9087007980698CD
:108B9000401CEFD02C461546FCF7F6FF0499401A0E
:108BA000059988420CD208980899491E0891002816
:108BB0002A46DED10590DCE72F461CE02F461AE05E
:108BC00028684168E02291434160412189006A6838
:108BD0008A420BD1A9680122D303994202D09202A2
:108BE000914203D101684022914301600020019924
:108BF000087001204870384609B0F0BDF0B583B068
:108C000016460D460446FCF7BFFF301A4719FCF71D
:108C1000BBFF0646214800684001000D78430290E2
:108C20002068806800210191000602D4019803B0F9
:108C3000F0BD20464830009003E0206880680006C0
:108C4000F4D5681CF9D0FCF79FFF801BB84207D20F
:108C500002980299491E02910028EED10746ECE7DE
:108C600020684168E02291434160412189006268A7
:108C70008A420BD1A1680122D303994202D0920209
:108C8000914203D101684022914301600020009984
:108C9000087001204870032003B0F0BDD000002010
:108CA00070470000F0B589B0FCF74AFA0146B548B4
:108CB00002F01CF96620B449085A8000B3490988BB
:108CC000814200D25CE11F20C04300903625B04CA9
:108CD000B0480890B0480690B04805905022B14F77
:108CE0000FE0921C0598001D05900698001D069047
:108CF0000898001D0890029C241D6D1C462D00D173
:108D00001FE1019220687F21CE053146FAF74EFA25
:108D1000002809D1F9F7ECFF1E21FAF73DFB0846C0
:108D20006430FAF78BFA20600795363D08980068A2
:108D30003146FAF73BFA00280AD1F9F7D9FF1E218C
:108D4000FAF72AFB08466430FAF778FA08990860BF
:108D5000032D0294049539D82068914F3946F9F7CC
:108D6000FDFF02F08FFC8F49FAF751F83F210D0605
:108D70002946F9F7F3FFFAF773FAF649079A8C18C0
:108D8000001D009EA055089800683946854FF9F7E8
:108D9000E5FF02F077FC3946FAF739F82946F9F78A
:108DA000DDFFFAF75DFA011D304610302154049AB8
:108DB000012A35D8A25D3F2A01D84022A255C9B266
:108DC0002C29774D54D82D21215451E02068744925
:108DD000F9F7C4FF02F056FC3946FAF718F83F21BC
:108DE0000E063146F9F7BAFFFAF73AFAD9490A2DD1
:108DF00026D8079A8918C01C009D48554C19089818
:108E000000686749F9F7AAFF02F03CFC3946F9F718
:108E1000FEFF3146F9F7A2FFFAF722FAC01C25E05F
:108E2000A25D079B382B00D085E0282A01D8292293
:108E3000A255C9B228295A4D1AD82921215417E020
:108E4000079A8918801C009D48554C19089800689D
:108E50005349F9F783FF02F015FC3946F9F7D7FFBC
:108E60003146F9F77BFFFAF7FBF9801C20744C4D73
:108E7000089800682946F9F771FF02F003FC3946AB
:108E8000F9F7C5FF3F210C062146F9F767FFFAF70E
:108E9000E7F9401CAF4F079AB854BE18069800680F
:108EA00029461546F9F75AFF02F0ECFB3D49F9F760
:108EB000AEFF2146F9F752FFFAF7D2F9801C03966C
:108EC00030743E46049C012C05D8715D402902D2C5
:108ED0004021344F06E0382D324F04D1715D2829EE
:108EE00001D829217155012C05D8C0B22C2802D8EF
:108EF0002D20039908740598006802F0C3FB3946D9
:108F0000F9F785FFFAF7ACF9801EC1B20A2900D83B
:108F10000A203221039A5054E0B2C01E0528019A5B
:108F200000D9DEE620488018009949000818163854
:108F30000088B052D5E6272A194D99D82820A05587
:108F400096E7134840242146F9F7FDFE11482146D3
:108F5000F9F7F9FE10482146F9F7F5FE0F482146CA
:108F6000F9F7F1FE00201049086048608860D84891
:108F70007821FAF763FC0A20FBF70AFFFCF7E8FE0A
:108F800009B0F0BD14130020301000202E0900207D
:108F90000C07002048030020CC060020940F00207E
:108FA0006F12833A0000A0411812002001490860A6
:108FB0007047C046BC110020014908707047C04688
:108FC00034080020F0B581B01C460D460646C11895
:108FD000571E5F433A46F9F79DFEF019294622468F
:108FE000F9F798FE01B0F0BD80B5074808210122CD
:108FF000FCF7C2FD80BDC04680B5034808210022B1
:10900000FCF7BAFD80BDC0460014005080B50520B5
:10901000000701221103FCF7AFFD80BD80B50520DC
:109020000007012109030022FCF7A6FD80BD000016
:10903000F0B581B0A44E307845490978884276D0A1
:10904000022813D0012853D0002870D1A0490889E4
:1090500030834868706163200A5C6420085C801873
:109060000F2866D8022A65D8501C63E0984FB88A4A
:109070003083386970613868FAF7EBF83649F9F7E8
:1090800003FFFFF7BBFB0446B0826320385C7083AC
:109090006520385CB083301D394636311022F9F72F
:1090A00039FE6225785D0090A0B2FFF793FB014680
:1090B000009802F037F885490880785D28282ED37B
:1090C0000020502103E0891C401C702927D03A1849
:1090D0004623D45C641CD454321813795B1C13717E
:1090E000C2B2D21E052AEED87A5A521D7A52EAE747
:1090F0007749C88930838889F0824889B0826320A3
:10910000085C70836520085CB083301D2631102216
:10911000F9F700FE74480021018001B0F0BD032082
:10912000C1010E48F9F70FFE0D480021017001B092
:10913000F0BD0F2070836520085CB083301D1631B0
:109140001022F9F7E7FD07480021017001B0F0BDDA
:10915000F40F002030100020000020418C0300207C
:1091600013120020C8060020F0B581B0564D2878B3
:1091700002280AD0012823D000285AD16888102854
:109180006ED30020287001B0F0BDA88AFFF722FB43
:10919000044668880F286AD80220287062204C494B
:1091A000085C214601F0BEFF484908804C48002178
:1091B000017041708170C1700171417101B0F0BDE9
:1091C00048480027078044480770454807704770A3
:1091D0008770C77007714771A88AFFF7FBFA0446CA
:1091E000414805882846FAF734F806463F492046A4
:1091F000F9F70DFE04463146F9F7AEFF3A4900286B
:1092000001D1681C08800888FAF723F80546204633
:109210002946F9F7A1FF00282B4E0ED170880F28A0
:109220000BD8718B814202D3B18B884214D20120BA
:1092300013E02FA001F09EFFFEE720462946F9F734
:10924000C3FF002811D070880F2824D8718B814269
:1092500021D3B18B88421ED30220307001B0F0BD03
:109260002148002101800120287001B0F0BD174D78
:109270002888002801D0401E28806227144EF05D07
:10928000214601F04FFF2888002807D002200E4910
:10929000087001B0F0BD377001B0F0BD0021009141
:1092A00009480170F05D214601F03CFF2880094823
:1092B0004021F9F748FD084800990170074801214D
:1092C000018001B0F0BDC046D40F0020CA060020C6
:1092D000301000203C0E002029100020D600002075
:1092E0009413002004130020880300200000C040D5
:1092F0003D3D3D3D3D3D3D3D3D204572726F7220FF
:109300005374617465203D3D3D3D3D3D3D3D3D0017
:1093100080B584B000210391029101910720009053
:109320006846FCF7F1FD002800D0FEE704B080BDE0
:1093300080B5FCF761FC00F027FB80BD07480168A1
:10934000074A0A40074909681143012252030A43A8
:1093500002600548054901607047C046041002409C
:109360000000FFFF040FFF1F08ED00E0002C0008C5
:109370000648704780B5002806D0002904D0024670
:10938000024804C0F9F7C6FC80BDC0469C1300200B
:1093900080B50248FDF7BCFF80BDC0469C08002098
:1093A000F0B58DB0F848FF260670F84C2670F84FDF
:1093B0007E807D8B00230C930B930A936220F549EA
:1093C000085C0122272801D8900700E0F2480790A6
:1093D00039780F20084002284AD0012862D000289E
:1093E0006CD1EE48F14903224023FFF7EBFDEC4836
:1093F0000178022901D8491C0170007801F00EFCA7
:109400003E7F788BB04200D2EFE1B000FB490858B4
:10941000E449F9F7A3FC02F035F9E349F9F7F7FC61
:109420000546B8190079F9F714FF01462846F9F7FF
:10943000AFFE002861D1761CF4B2788BA04200D236
:10944000D3E1A000ED490858FC49F9F787FC02F088
:1094500019F9FB49F9F7DBFC054638190079F9F7EA
:10946000F8FE01462846F9F785FE0028E3D145E0DD
:10947000099504930092391DE048FEF721FFDC4D69
:109480002870DD494631DE48FEF71AFF2070297842
:10949000FF2817D0FF29099D35D0DA48049A0280A9
:1094A00079803DE0391DD548FEF70AFFD0490870A4
:1094B000FF2800D199E178800DB0F0BDE1A002F065
:1094C000B3F9FEE7FF29099D22D0CE480188491C47
:1094D000018088B2F9F7BDFE0446B88AFFF77AF931
:1094E0008121C905F9F793FC2146F9F75FFE0028B1
:1094F00014D0BF480078788011E03446BC4806702C
:109500007C800DB0F0BDBA490978FF2900D136E161
:109510007E80BC480188491C018000E07E80049A5E
:10952000B9480078002800D05FE1B84882704270E6
:109530000270B7480270B74800780F2802D8401C64
:10954000B44908707888102800D24EE1092D03D361
:109550000920042805D234E1681CC0B2042800D2D6
:109560002FE10321AD4E069101900CE0A748007851
:10957000C10700D11CE10698401C0690C1B20198B9
:10958000884200D81DE103914021A348F9F7DBFB95
:10959000049931607160B160F160316171619D4821
:1095A000027810200292801AC0B205900F28084657
:1095B00009912BD80698C0B2059B9900964A561877
:1095C000062159430818800095490F180C3F5C1C70
:1095D000002009900890388800B2308002217D5E1A
:1095E0007580F9F72BFE01460998F9F7B7FB09904A
:1095F0002846F9F723FE01460898F9F7AFFB18371C
:10960000621C361DE1B210291446E3D1099F0646BB
:10961000029810281BD100247F4D285F0001F9F724
:109620000DFE3946F9F7EBFBF9F71AFE28532D1911
:109630000220285E0001F9F701FE3146F9F7DFFB51
:10964000F9F70EFE6880241D402CE5D137E005991E
:109650000F2934D83446F9F7FCFD0546384629462B
:10966000F9F712FC099030462946F9F70DFC074638
:10967000059A900068490E18541C0220305EF9F7D4
:10968000DDFD3946F9F7BBFB8321CD052946F9F706
:10969000BEFBF9F7E5FD7080308800B2F9F7CEFD2A
:1096A0000999F9F7ACFB2946F9F7B1FBF9F7D8FDB1
:1096B0003080601C361DE1B210290446DDD1002740
:1096C00001245848544D29463A46234600F012FAE0
:1096D0000A35524EF15BE243AA5E5243120A8918E0
:1096E0002A8812B25243120A8918F1532D1DBF1C49
:1096F000182FEFD14C480C904C480B904C480A90D6
:109700000AA900270B2330463A4601F0ACFB039828
:109710004000394940185021405A0A30F18A8842A5
:1097200000D223E709913E4602E0BF1C102F11D062
:109730003A48C0198088F9F78CFD01463046F9F7A0
:109740000DFB05463B4E3146F9F714FD0028ECD1E0
:109750002E46EAE707983146F9F759FB0546099E78
:109760003046F9F776FD102E2C4E00D203E7014665
:109770002846F9F7FFFC002800D0F7E6FBE6214970
:10978000049A0A807880CBE6241200200613002079
:10979000D40F0020301000200000204028120020AC
:1097A000291000206F12833A0000A041540F0020BE
:1097B0001649069A4A70204308700AA8C07A801C8D
:1097C00088701D48114C022203232146FFF7FAFB43
:1097D00001F0DCFA00280749009A0D4B05D04888B3
:1097E000102802D31A70607848800DB0F0BDC046D2
:1097F00024120020D40F002030100020540F00202D
:109800003C0E00200413002013120020141200202C
:10981000C8060020291000207C0E0020BC0E00206D
:109820008C03002020BB000808090A0B040506076A
:10983000000102030000E040941300206F12833AFD
:109840000000A0413D3D3D3D3D3D3D3D3D2045723B
:10985000726F72205374617465203D3D3D3D3D3D06
:109860003D3D3D0D00000000B0B521480F490022EC
:109870000F4B104C2546103D056043608260C1606F
:10988000026142618261FDF7C7FC002800D0FEE75B
:1098900020680121884320601324002120460A46C5
:1098A000FCF73AFA2046FCF72BFAB0BD2F75000002
:1098B000BF120000102000400D48006800214162E6
:1098C0007047C04610B5094C2078002807D10848D9
:1098D000FDF70EFD002800D0FEE7012020700848AB
:1098E000016801220A43026010BDC046DC08002066
:1098F0009C080020024801680122914301607047E2
:1099000000200040F0B51149C88A00281CD0C88A40
:10991000497E8A000023002905D15B1CDDB2A842E4
:1099200012D90029F9D0DDB248266E43084CA5199A
:109930000026AF19BC8864BAAC53FC8864BA7C803A
:10994000361DB242F5D1E8E7F0BDC046D40F002085
:109950000806002010B5564C00200A490C227D2331
:10996000DB020AC420606060A060E2602061083C05
:109970002046FDF7E5FD2068C16820220A43C26049
:1099800010BDC046004400404A48016800290AD082
:1099900049490A68521C0A600B2A04D3002101605D
:1099A0000148012101607047C4130020F0B581B067
:1099B000044601214A03006803699343E2681A439D
:1099C00002612269C3682A4D1D40A368134362697E
:1099D0001A432A43C260CD024169A943E669314373
:1099E00041610321090242698A43A169114341612E
:1099F000FCF78AFB0146192048436168AE421AD140
:109A00004900F9F7A9FC064664273946F9F7A4FC92
:109A10000546194868438019C00032303946F9F7C5
:109A20009BFC0721014040001F2212010240280137
:109A30001018401817E08900F9F78EFC06466427D5
:109A40003946F9F789FC05460A4868438019000140
:109A500032303946F9F780FC0F210140F0220240F4
:109A60002801101840182168886001B0F0BDC04678
:109A7000F3E9FFFF9CFFFF0F9CFFFF1F80B501F084
:109A80002BF9002802D00348006880BD00F004F8DC
:109A900080BDC0460444004080B50548FDF73CFD4C
:109AA00004480121016004480021016080BDC046D6
:109AB000E00800205414002058140020F0B50029BC
:109AC00016D000235C00155BAD086D00465B1419D1
:109AD0006488A4086400075B4753065345196E88E1
:109AE000041967886F8066809B1C9BB28B42E9D308
:109AF000F0BD000070B51E460C4605460188012ADF
:109B00000FD1FF291DDD3048814228DD01200203ED
:109B100091423DD0C202914235D08002814237D07D
:109B20004AE0FF2914DD2848814220DD012002039C
:109B300091423CD0C202914234D08002814236D060
:109B40003AE03F291BDC102922D020291BD033E02A
:109B50003F2923DC10292AD0202923D02CE0012002
:109B60000202914214D0400281420CD024E0012034
:109B7000020291421BD04002814213D01CE04029D6
:109B800006D0802918D16A68204600F01FF813E03B
:109B90006A680123204600F075F90DE0402906D0DF
:109BA000802909D16A68204600F08CF804E06A68D0
:109BB0000123204600F044FC002E04D0AA68A989A5
:109BC0002046FFF77BFF70BDFF030000F0B58DB0AE
:109BD00016460A4605464C08049162D0A0000C9037
:109BE000029529460196354603940B9402242B5F77
:109BF0000C9A885E401007900E8836B27610089650
:109C000086197608288806900E800E5F77100597D3
:109C100088180A90045F6610B81B09901F464743D6
:109C20003F0C0898079A841A069802B210466043BF
:109C3000000CC01B0C9FC853059830184008488082
:109C40006343180C099B5A43120C10180A9A50804F
:109C50000B9C091D2D1D641EC7D10227029D28469D
:109C6000039C2146019E32463B4600F00BF90498C6
:109C700040002818214632463B4600F003F9002CEC
:109C80001ED0E8884000E880A8884000A880688846
:109C9000400068802888400028800835641EF0D184
:109CA0000EE002272846214632463B4600F0EAF8FD
:109CB000049840002818214632463B4600F0E2F85E
:109CC0000DB0F0BDF0B58DB016460A4605464C08FD
:109CD000049162D0A0000C90029529460196354669
:109CE00003940B9402242B5F0C9A885E401007901B
:109CF0000E8836B27610089686197608288806905F
:109D00000E800E5F7710059788180A90045F661022
:109D1000B81B09901F4647433F0C0898079A841ABE
:109D2000069802B210466043000C38180C9FC853C6
:109D300005983018400848806343180C099B5A4323
:109D4000120C101A0A9A50800B9C091D2D1D641EBE
:109D5000C7D10227029D2846039C2146019E324618
:109D60003B4600F06DFB049840002818214632461F
:109D70003B4600F065FB002C1ED0E8884000E880E0
:109D8000A8884000A8806888400068802888400033
:109D900028800835641EF0D10EE0022728462146AF
:109DA00032463B4600F04CFB049840002818214600
:109DB00032463B4600F044FB0DB0F0BDF0B581B03B
:109DC0000D4606460092940843D030680146F9F7E4
:109DD0001EF8074670680146F9F719F8014638463B
:109DE000F8F7BCFF01F030FD2860B0680146F9F7D4
:109DF0000EF80746F0680146F9F709F801463846BB
:109E0000F8F7ACFF01F020FD686030690146F8F713
:109E1000FEFF074670690146F8F7F9FF014638462C
:109E2000F8F79CFF01F010FDA860B0690146F8F753
:109E3000EEFF0746F0690146F8F7E9FF01463846AC
:109E4000F8F78CFF01F000FDE86010352036641E45
:109E5000BBD10320009C044012D030680146F8F7C3
:109E6000D6FF074670680146F8F7D1FF014638462D
:109E7000F8F774FF01F0E8FC01C50836641EECD168
:109E800001B0F0BDF0B5A2B00C2425465D4311959C
:109E90000A918908039427464F439C001094069327
:109EA000DB000F938B001E93CB0019930090209240
:109EB0001F9204921D9202911A9718911E99415E69
:109EC0008910C25F9210531801498B4206DC01E0F1
:109ED0000080FFFF004B01E00080FFFF01498B4243
:109EE00003DB01E0FF7F00000B465908199D425F2C
:109EF0009410028812B2921016941592A21813921E
:109F00005408091901800226815F8A1041191791AE
:109F1000895F89101B9214918C181E994118129117
:109F20008D5FAD10C21921961C92965FB6107519FF
:109F3000EA4EB54200DCE94D6608E94FBD4200DB60
:109F4000E74D6F08BE194680641BE44FBC4200DC3D
:109F50003C46E34EB44200DB3446219D1F9A555FD8
:109F6000139AD21ABA4200DC3A462B466343B242F5
:109F700000DB32461F9E368836B237465743FB1AFF
:109F80001F0C1E9BC15E1391C75274435543621947
:109F9000140C219A12998A5E4C801B99149BCD1A3D
:109FA000CE4FBD4200DC3D46CD4EB5421A9C00DB93
:109FB000354613998910035F9B10C91AB94200DC1A
:109FC0003946B14200DB314614914919B94200DCEF
:109FD0003946B14200DB3146219B209CE45E13945C
:109FE00092101C9CE35E9B10D21ABA4200DC3A46E7
:109FF000B24200DB32461B92169A159CA21ABA4254
:10A0000000DC3A461695B242139B00DB32461B9C9D
:10A01000151BBD4200DC3D461C464C43B54200DBEF
:10A020003546209E37883EB237466F433C1B240C92
:10A03000199FC45371436B435918090C179C6180D5
:10A040001699149C091BFD4CA14200DC2146FA4DD7
:10A05000A94200DB2946219C1D9E345F1B9B9A1858
:10A06000F64B9A4200DCF54A1B9023464B43AA422A
:10A0700000DB2A461D9F3D882DB22E465643F31A1B
:10A080001B0C1A981B9E3352694354436118090CE8
:10A090001C9A51801099209A521820920F991F9A59
:10A0A00052181F9211997F181D9707463046301D90
:10A0B0001899491E00D000E70A9B1809142B00D2FA
:10A0C00010E1DD4D1946029A0191039E4643C100FD
:10A0D000209181001F910C9291000B910290401EE3
:10A0E000059006988000069000210098099008913C
:10A0F0001A960791994200D3DCE00620089A504353
:10A10000910052004000049B1C5E0F9452009C5E24
:10A110001D9449005C5E0E94219C2043185E1C90A7
:10A120002243985E1B902143585E0D900999079831
:10A130001990885F1F9A8A5E1018A84200DB284693
:10A14000BE4B984200DC1846209A8C5E0A8812B2F8
:10A15000189417921219AA4200DB2A4640109A421C
:10A1600000DC1A46521005461492801840080880F8
:10A170008819219A1E90805E1F9C0C191594A25E6E
:10A180001718AD48874200DBAB4F9F4200DC1F46EB
:10A1900021980C5E209A8A181692105E13941290E1
:10A1A0002218A548824200DBA34A7C109A42284626
:10A1B00000DC1A4653101A1B0D9F3D46554311945F
:10A1C000149C201A0E9E34464443641B240C1094A5
:10A1D0001F9D4C5F1494109C4C53119CE3185B081A
:10A1E0004B80724378431018000C219A159CA35E93
:10A1F00060801398129A801A8F4EB04200DB30466E
:10A200008E4A904200DC8D481A9A8A5E149CA41AE9
:10A21000B44200DB3446894A944200DC874C219AE0
:10A220001E9DAA5E9D1AB54200DB354640106210A5
:10A23000824B9D4200DC1D46159014921018189A0E
:10A24000179FBA1AB24200DB32461B9F47436E107B
:10A250009A4200DC1A465210951B1D9B6B43DB1B78
:10A260001B0C209FCB53159B149C1B1B1C9C5C43FD
:10A27000B2180F9F3E465643341B240C1A9E8C5333
:10A280001D9C60431B9C65432818000C169C608035
:10A290007B431C984243D018000C1E9A50800B98A8
:10A2A00009180C98199A121810460A9B9A42624D86
:10A2B00000D23DE706980899091808910998001DF1
:10A2C00009900799491C0598814200D811E7029A24
:10A2D0009008019CA108502C05D3F5E60080FFFFF3
:10A2E000FF7F0000029A039941430391991A189144
:10A2F00081002191C700900016900098841C0021D5
:10A30000C84346004C4D029217971E91E0191D90CC
:10A31000805FA15F1C901B910918A94200DB2946B0
:10A320004648814200DC4549039820182090805F10
:10A33000219AA218935F1818A84200DB28464B10F8
:10A340003E49884200DC3D4841101993CD18E05F3A
:10A350001F900398275E2198235E2088A553DF195C
:10A36000354B9F4200DB1F46344B9F4200DC334F8E
:10A3700003B21F981A931D182F48854200DB2E4DFB
:10A3800078102E4B9D4200DC2C4D6D10431923801C
:10A39000199B5F1A915F19912199635E9753281A4F
:10A3A00060521C981B990A1A23498A4200DB0A460C
:10A3B00022488242179F00DC204A0398205E181A28
:10A3C000884200DB084652101C49884200DC1B48CA
:10A3D00043101C92D01A20998D5F1D9988531998AB
:10A3E000411B154DA94200DB29463A4613488142DC
:10A3F00000DC12491F981A9F381AA84200DB284631
:10A4000049100E4DA842174600DC0C4840100D18AC
:10A41000E5531C9A9A18209B9A53401A039960524C
:10A4200016982418029A1E99891818988142024D8C
:10A4300000D86AE722B0F0BDFF7F00000080FFFF78
:10A44000F0B5A2B00C2425465D4311950A91890808
:10A45000039427464F439C0010940693DB000F9310
:10A460008B001E93CB001993009020921F920492B0
:10A470001D9202911A9718911E99415E8910C25F30
:10A480009210531801498B4206DC01E00080FFFF67
:10A49000004B01E00080FFFF01498B4203DB01E03C
:10A4A000FF7F00000B465908199D425F94100288F7
:10A4B00012B2921016941592A21813925408091908
:10A4C00001800226815F8A1041191791895F8910E6
:10A4D0001B9214918C181E99411812918D5FAD102A
:10A4E000C21921961C92965FB6107519EA4EB542B4
:10A4F00000DCE94D6608E94FBD4200DBE74D6F081F
:10A50000BE194680641BE44FBC4200DC3C46E34E6F
:10A51000B44200DB3446219D1F9A555F139AD21A2C
:10A52000BA4200DC3A462B466343B24200DB324675
:10A530001F9E368836B237465743DB191F0C1E9BC9
:10A54000C15E1391C75274435543621B140C219A88
:10A5500012998A5E4C801B99149BCD1ACE4FBD4236
:10A5600000DC3D46CD4EB5421A9C00DB35461399C2
:10A570008910035F9B10C91AB94200DC3946B14209
:10A5800000DB31461491691AB94200DC3946B14208
:10A5900000DB3146219B209CE45E139492101C9CAE
:10A5A000E35E9B10D21ABA4200DC3A46B24200DBAC
:10A5B00032461B92169A159CA21ABA4200DC3A4601
:10A5C0001695B242139B00DB32461B9CA518BD4278
:10A5D00000DC3D461C464C43B54200DB3546209E20
:10A5E00037883EB237466F433C19240C199FC45339
:10A5F00071436B43C91A090C179C61801699149C0E
:10A600006118FD4CA14200DC2146FA4DA94200DB55
:10A610002946219C1D9E345F1B9BD21AF64B9A4201
:10A6200000DCF54A1B9023464B43AA4200DB2A4636
:10A630001D9F3D882DB22E465643F3181B0C1A98C9
:10A640001B9E335269435443091B090C1C9A5180C9
:10A650001099209A521820920F991F9A52181F92FF
:10A6600011997F181D9707463046301D1899491ECD
:10A6700000D000E70A9B1809142B00D210E1DD4D31
:10A680001946029A0191039E4643C1002091810020
:10A690001F910C9291000B910290401E059006981C
:10A6A0008000069000210098099008911A96079161
:10A6B000994200D3DCE00620089A504391005200F2
:10A6C0004000049B1C5E0F9452009C5E1D94490048
:10A6D0005C5E0E94219C2043185E1C902243985E81
:10A6E0001B902143585E0D90099907981990885F37
:10A6F0001F9A8A5E1018A84200DB2846BE4B98427B
:10A7000000DC1846209A8C5E0A8812B218941792C0
:10A710001219AA4200DB2A4640109A4200DC1A466F
:10A720005210054614928018400808808819219A12
:10A730001E90805E1F9C0C191594A25E1718AD48E0
:10A74000874200DBAB4F9F4200DC1F4621980C5E26
:10A75000209A8A181692105E139412902218A54817
:10A76000824200DBA34A7C109A42284600DC1A464B
:10A7700053101A1B0D9F3D4655431194149C201AEB
:10A780000E9E344644432C19240C10941F9D4C5F9C
:10A790001494109C4C53119CE3185B084B8072433B
:10A7A0007843101A000C219A159CA35E60801398C0
:10A7B000129A801A8F4EB04200DB30468E4A904289
:10A7C00000DC8D481A9A8A5E149CA41AB44200DBFD
:10A7D0003446894A944200DC874C219A1E9DAA5E29
:10A7E0009D1AB54200DB354640106210824B9D42F7
:10A7F00000DC1D4615901492801A189A179FBA1AF9
:10A80000B24200DB32461B9F47436E109A4200DC87
:10A810001A465210B5181D9B6B43DB191B0C209F69
:10A82000CB53159B149CE3181C9C5C43921B0F9FFD
:10A830003E4656433419240C1A9E8C531D9C60438B
:10A840001B9C6543401B000C169C60807B431C983E
:10A850004243981A000C1E9A50800B9809180C98C5
:10A86000199A121810460A9B9A42624D00D23DE78F
:10A8700006980899091808910998001D09900799E8
:10A88000491C0598814200D811E7029A9008019C62
:10A89000A108502C05D3F5E60080FFFFFF7F0000E4
:10A8A000029A039941430391991A189181002191C9
:10A8B000C700900016900098841C0021C8434600F1
:10A8C0004C4D029217971E91E0191D90805FA15F79
:10A8D0001C901B910918A94200DB29464648814279
:10A8E00000DC4549039820182090805F219AA21827
:10A8F000935F1818A84200DB28464B103E49884257
:10A9000000DC3D4841101993CD18E05F1F9003987B
:10A91000275E2198235E2088A553DF19354B9F427F
:10A9200000DB1F46344B9F4200DC334F03B21F98BD
:10A930001A931D182F48854200DB2E4D78102E4BA0
:10A940009D4200DC2C4D6D1043192380199B5F1A2A
:10A95000915F19912199635E9753281A60521C9850
:10A960001B990A1A23498A4200DB0A46224882427E
:10A97000179F00DC204A0398205E181A884200DBEB
:10A98000084652101C49884200DC1B4843101C92A8
:10A99000981820998D5F1D9988531998411B154D62
:10A9A000A94200DB29463A461348814200DC12499D
:10A9B0001F981A9F381AA84200DB284649100E4DEE
:10A9C000A842174600DC0C484010451AE5531C9A73
:10A9D000D21A209B9A53081803996052169824188B
:10A9E000029A1E99891818988142024D00D86AE788
:10A9F00022B0F0BDFF7F00000080FFFF0148002172
:10AA000001707047300C0020B5480021017070477C
:10AA1000F0B583B07E4C294D2560089C002A19D0E2
:10AA2000A34211D2E11A9A008018DA00AA1803880A
:10AA30001BB29B0213600223C35E9B025360491E3C
:10AA4000001D08320029F2D11D488021F8F77BF95A
:10AA500003B0F0BDA34202912DD2E21A0A2402995A
:10AA6000611A00919E008019DE00154B9B19AD19EB
:10AA70002E68374602990F41F61B07883FB2BC0289
:10AA800000998F40BE192E60A41B1C600224045F35
:10AA9000A60201968C4069680F46029E3741C91B89
:10AAA00061186960019C611A5960521E001D0833CB
:10AAB0000835002ADCD103B0F0BDC046B00A002042
:10AAC000B0090020F0B583B0514D244C2C60002A11
:10AAD00016D0012A40D1002B0CD0018809B289027E
:10AAE00021600221415E890261605B1E001D083405
:10AAF000002BF2D11A488021F8F725F903B0F0BDF8
:10AB0000002B029128D00A220299511A0091134C6D
:10AB1000134D2668374602990F41F61B07883FB24E
:10AB2000BA0200998F40BE192660921B2A60022249
:10AB3000825E960201968A4061680F46029E374106
:10AB4000C91B51186160019A511A69605B1E001D92
:10AB500008350834002BDCD103B0F0BD300B0020E9
:10AB600030090020F0B583B0294C2A4D2560089C9F
:10AB7000002A19D0A34211D2E11A9A008018DA00F3
:10AB8000AA1803881BB29B0213600223C35E9B02B8
:10AB90005360491E001D08320029F2D11E48802151
:10ABA000F8F7D1F803B0F0BDA34202912DD2E21A1A
:10ABB0000A240299611A00919E008019DE00164B4A
:10ABC0009B19AD192E68374602990F41F61B07886D
:10ABD0003FB2BC0200998F40BE192E60A41B1C60BE
:10ABE0000224045FA60201968C4069680F46029E0B
:10ABF0003741C91B61186960019C611A5960521E76
:10AC0000001D08330835002ADCD103B0F0BDC04672
:10AC100000130020B00B0020300A0020F0B587B0F0
:10AC2000022834D30546F8F714FB0446194F44377D
:10AC3000684201900E20C0430690002005940390C6
:10AC40008600154880592146F8F71EF90546124836
:10AC5000855180190290069E0E360497019C386833
:10AC60000599F8F711F901462846F8F777F80546EF
:10AC7000069880003F18761EB442F0D10298056015
:10AC8000049F3F1D0398401C0E28059CD7D107B098
:10AC9000F0BDC04628120020540F002080B582B0BD
:10ACA0000190974801A90122024BFCF7DFFC0198B3
:10ACB00002B080BDFFFF000080B503464820484336
:10ACC00004490818E849497E8A0008321946F8F70D
:10ACD00021F880BD08060020014800787047C04672
:10ACE000101300206F2806DC2F280CD06D280CD103
:10ACF000094908467047772809D0702805D1D52022
:10AD00004101084670474320010208467047014947
:10AD1000084670470F360000C0E80000FDF78CFBC6
:10AD2000F8F7F6FFF9F716FDFCF7BCFF6420F8F71B
:10AD300055FDFCF7D9FFFDF70FFC7D200001F8F76A
:10AD40004DFD00F003FA084840884004000CFDF770
:10AD500031FE0648FAF748FFFDF7E2FBF8F7E4FF9B
:10AD6000FAF734F9F8E7C046E0070020AC06002007
:10AD700010B50C46014603482246F7F7CBFF0248C0
:10AD8000046010BD340D0020B40D002001221249D2
:10AD90008B5C0020002B1CD0D21C072AF8D10A792A
:10ADA0004B789A1AD317D2185A40012A11DC4B79E2
:10ADB00008221846083800D8D01A8B781946083966
:10ADC00000D8D11A081AC11740184840022801DBE0
:10ADD000002070470120704794130020F0B587B021
:10ADE0000D46014658000C180194541E06949A42D0
:10ADF0000293049526DA085A0590AE189D1A500061
:10AE00000C180A46039111E0069F7F1C7800101869
:10AE1000214600F049F804980697C019314600F021
:10AE200048F8039AA41C761C6D1E0CD02088059946
:10AE30008842E9D3F6D102980499085C31788142BE
:10AE4000E2D3EFE70A460698441C60001018019907
:10AE500000F02AF80298049A1118101900F029F845
:10AE6000204607B0F0BDF0B581B09A4214DA17461B
:10AE70000E4605460093284631463A46009BFFF7AA
:10AE8000ADFF0446431E284631463A46FFF7EBFF26
:10AE9000009B671C9F42EEDB01B0F0BD0148012121
:10AEA00001707047300C002002880B8803800A80F4
:10AEB000704702780B7803700A707047B0B5084D80
:10AEC000286801280BD1074C2046FCF71DFB0146E2
:10AED000054801602068FFF74BFF00202860B0BDE7
:10AEE000C4130020CC130020C813002080B50A46EC
:10AEF00001467D20C3000248FCF7B8FB80BDC04678
:10AF0000E00800200D2807D0442809D13F20800206
:10AF100001401143084670477F2040020140114321
:10AF200008467047F0B587B006A80021018005915A
:10AF300004910391029101914B4C26780F252E40EC
:10AF4000638B022E06D14C4801784848FF2910D067
:10AF500002460FE06088454A002E11D110280FD319
:10AF60004348444A1170016041608160C1600161E1
:10AF700072E0424A42490978FF2900D102466088BE
:10AF80000F283BD8022E06D0002E08D1462141437F
:10AF900006A8018026E03B4909780129F6D0A18B5B
:10AFA000884205D100280ED106A82321018019E08E
:10AFB000591CC9B2491E814205D10F2803D106A8E8
:10AFC000324901800EE08300D158D2185368121F15
:10AFD0001268FCF7C9FC2C49F7F719FFF8F740F99C
:10AFE00006A9088023480178092901D8491C017065
:10AFF0001F4806A90A220223FDF7E4FF2078FAF78A
:10B000007FF900280FD01B482178102902D0017841
:10B0100000290CD1164A0021017011605160916025
:10B02000D160116118E013480178002917D0104849
:10B0300001AA48C848C2C8C8C8C220782840012808
:10B0400002D106A8018807E00A20401A400001AAA0
:10B050001018FCF79DFD0146084607B0F0BD0CA096
:10B0600000F0E2FBFEE7C046D40F0020540F0020A2
:10B07000141000209A130020241200203C0E0020FF
:10B0800006130020C806002000008C421A040000AD
:10B09000E697A0E69C89E69588E8B79DE7A6BBE51C
:10B0A000B9B3E6BB91E695B0E68DAEEFBC810D007D
:10B0B000B0B502780F211140022915D0012927D1FE
:10B0C000041D174D2946263110222046F7F722FE8F
:10B0D0006320285C02281AD80020215C891F215493
:10B0E000401C0628F9D112E0041D0D4D29463631C9
:10B0F00010222046F7F70EFE6320285C022806D8AF
:10B100000020215C491F2154401C0628F9D1B0BD04
:10B11000001D034916311022F7F7FCFDB0BDC046F3
:10B120003010002010B50C460F2803D88120C1052F
:10B13000204603E00C38F8F781F82146F7F767FE60
:10B14000F8F78EF8022800D8022010BD80B5054817
:10B1500000780322424304480449054BFBF766FD8F
:10B1600080BDC04611130020C0110020380200200D
:10B17000881300000FB410B503A9044B044A0298C9
:10B1800000F046F810BC08BC04B018479DAC00089D
:10B19000C40000202021020C01D010211046020A18
:10B1A00001D010460839020901D01046091F820853
:10B1B00001D01046891E420801D0881E7047081A27
:10B1C000704710B57F200021C005F7F75DFE10BD68
:10B1D00010B50121F8F7ADF910BD10B500210846F2
:10B1E000F7F752FE10BD02E008C8121F08C1002A7E
:10B1F000FAD170477047002001E001C1121F002AF8
:10B20000FBD170470149086070470000C80000206A
:10B21000FFB591B00F460546002606E025280AD066
:10B22000149A139990476D1C761C28780028F5D144
:10B23000304615B0F0BD002400940121F34A029479
:10B2400000E004436D1C2B780846203B98401042D8
:10B25000F7D128782A280ED0022128780246303AE1
:10B26000092A15D8009A0A235A43303A80180C4309
:10B270006D1C0090F1E701CF0090002805DA012055
:10B2800040030443009840420090022004436D1C98
:10B2900028782E2815D10420044368786D1C2A28AC
:10B2A0000AD101CF6D1C02900BE002990A22514392
:10B2B000303940186D1C0290287801463039092930
:10B2C000F3D928786C2810D006DC4C281AD06828CE
:10B2D0000ED06A2817D104E0742813D07A2812D12E
:10B2E00010E00120400504430CE00121090501E0C4
:10B2F000032109050C436978814203D1012000052F
:10B3000024186D1C6D1C287803906E281ED00CDC50
:10B31000632831D004DC00288AD0582811D1B2E04B
:10B3200064287BD069280CD178E073282DD004DC08
:10B330006F2870D0702804D1A7E075286CD07828C9
:10B340006BD0149A13999047761C62E06002400F0C
:10B35000022807D003280AD0042838680AD00660DB
:10B360003F1D56E03868F11706604160F8E738681D
:10B370000680F5E70670F3E7387869460874002020
:10B38000487404A80390012003E03868039000206B
:10B39000C0433F1D61070FD5002101E00199491C01
:10B3A000029A0191914213DA8142F7DB019A0399E3
:10B3B000895C0029F2D10BE0002101E00199491CD0
:10B3C00001918142FADB019A0399895C0029F5D148
:10B3D00001990098139A401A00902146149B00F09E
:10B3E0003BF901998019461807E003980399007802
:10B3F000491C0391149A139990470198401E01909B
:10B40000401CF2D12146149B139A009800F014F9C5
:10B4100086196D1C09E741E033E034E00A20002181
:10B42000049005916002410F022905D001CFC21797
:10B430009446032905D007E0FF1DFF08FF0003CF56
:10B4400006E000B2C2179446042902D140B2C117E7
:10B450008C4600226146944506DA0A4600214042A5
:10B4600091418C462D2102E0210504D52B216A460D
:10B470001176012103E0E10701D02021F7E70191D6
:10B4800054E00A200BE0102009E010200490002175
:10B490000420044308200591029003E008200021C5
:10B4A000059104906002410F022905D001CF0022CE
:10B4B0009446032906D006E0FF1DFF08FF0003CFD6
:10B4C0008C4603E080B2042900D1C0B20021019172
:10B4D00021072BD50399702906D0049A1021059BCA
:10B4E0004A401A4305D00EE040216A4611760121F8
:10B4F00008E06146014306D030216A46117603997F
:10B50000517602210191049A0821059B4A401A4371
:10B510000CD16146014301D1610707D530216A464C
:10B520001176012101910299491E0291039958292E
:10B5300004D037A103910FA90F910DE039A1F9E7CC
:10B540006146059B049AF7F74FFF039B8C469B5C73
:10B550000F9A521E0F92137061460143F0D10F985B
:10B5600007A9081A20300390600704D501200004C1
:10B570008443029801E0012002900399884201DD92
:10B58000401A00E000204118029001980918009824
:10B59000401A0090E00306D42146149B139A0098A9
:10B5A00000F05AF886190020049008E006A9085C0B
:10B5B000149A139990470498401C761C04900199A2
:10B5C0008842F3DBE0030CD52146149B139A0098C4
:10B5D00000F042F8861904E0149A3020139990473D
:10B5E000761C0299481E02900029F5DC08E00F98AD
:10B5F0000F990078491C0F91149A13999047761C63
:10B600000399481E03900029F1DCFBE6092801009C
:10B6100030313233343536373839616263646566C8
:10B62000000000003031323334353637383941428A
:10B630004344454600000000F8B5044600251E4678
:10B640001746880404D405E039462020B0476D1C15
:10B65000641EF9D52846F8BDFFB50446002581B023
:10B660001E46C80301D5302700E02027880404D5F2
:10B6700005E038460399B0476D1C641EF9D528468D
:10B6800005B0F0BDF8B50121C9057F220026411A99
:10B69000120691427ED20121C9044118CA15012324
:10B6A00041021B07C9184D0F7F217F3A2B05C905A1
:10B6B000B6185C18D205871A3046284345D0214673
:10B6C0003846F7F74BFB009021463846F7F797FBD3
:10B6D0000099F7F7D9FB07460146F7F798FB45496C
:10B6E0000090F7F794FB4449F7F738FB04463846D7
:10B6F0000099F7F78CFB2146F7F789FB04463046A3
:10B70000F7F79CFD06463D49F7F781FB3C49AD0044
:10B7100079444959F7F722FB2146F7F71FFB044606
:10B7200038493846F7F773FB2146F7F717FB04460D
:10B7300030463549F7F76BFB344979444959F7F7F7
:10B740000DFB2146F7F70AFBF8BD3846F7F757FB24
:10B7500005462F49F7F75BFB2E49F7F7FFFA294615
:10B76000F7F755FB2C49F7F7F9FA2946F7F74FFB9E
:10B770002A49F7F7F3FA044629460846F7F747FB44
:10B780002146F7F744FB044625492846F7F73FFBD7
:10B79000214600E00AE0F7F7E1FA0446214928468D
:10B7A000F7F735FB2146F7F7D9FAF8BDFF2241003C
:10B7B0001206914202D9FFF70BFDF8BDFF22D20518
:10B7C0009042FAD01402A04205D90120FFF71AFDD9
:10B7D000FFF703FDF8BD410005D01626F6431721FB
:10B7E000F7F7A7FE57E70220FFF70CFDFFF7E9FC8C
:10B7F0006040F8BDDE02323E3B3D943EFC849A360A
:10B8000080010000D95B5E3F00209A3E36010000B7
:10B81000924FA93D7279DEBD2D3E143ED85B5EBECF
:10B82000157B4B3C0000D83E10B5044601E0FFF705
:10B8300035FA2078641C03490028F8D10A20FFF764
:10B840002DFA10BDC400002070B50546F7F77DFE47
:10B8500041000446FF204908C005411AC90F07D01E
:10B8600069004908401AC00F02D10120FFF7CAFC45
:10B87000204670BD000000000080513D0070C63DB4
:10B8800000900D3E0050343E00E0573E00D0783E20
:10B8900000C08B3E000000000AD6A936431C8C373E
:10B8A000658F7338832DA236121D1F38B3756F381C
:10B8B000D2535A380080000001000200000000004E
:10B8C00000093D0000127A000024F4004086510176
:10B8D00000366E010000000031780008CD770008C6
:10B8E0000000000000000000000000000000000058
:10B8F0000000000000000000000000000000000048
:10B90000010000000200000003000000040000002D
:10B910000600000007000000080000000900000009
:10B920000000000000000000000000000000000017
:10B9300001000000020000000300000004000000FD
:10B9400000093D0000127A000024F40040865101F5
:10B9500000366E0100093D0000093D0000093D0070
:10B96000430024134400017C450000004600F4011C
:10B97000470000104800280A490000204A00A3029E
:10B980004B0000004C0065044D0000004E0001001B
:10B990004F0000005000EE0251001C005200D9FD83
:10B9A0005300155054005655550000005600121211
:10B9B0005700FFFF580051BA5D0001065E0032FFDC
:10B9C0005F00162D61000801620088006300080115
:10B9D0006400880065000000660000006700000049
:10B9E0006C0060C66D00C0EE6E00D8036F0003559A
:10B9F0007000A03E7600010077000F0606003401BB
:10BA0000020036000B00360C0D0001403E00111004
:10BA10003A004886FF00FFFF000000000000000021
:10BA20000000000000000000000000000000000016
:10BA30000000000000000000000000000000000006
:10BA400000000000000000000000000000000000F6
:10BA500000000000000000000000000000000000E6
:10BA600000000000000000000000000000000000D6
:10BA700000000000000000000000000000000000C6
:10BA800000000000000000000000000000000000B6
:10BA900000000000000000000000000000000000A6
:10BAA0000000000000000000000000000000000096
:10BAB0000000000000000000000000000000000086
:10BAC00000000000000000007200D00241000440AD
:10BAD000000000200100648D40000702FF00FFFF0E
:10BAE00000000000000000001C0FFF1F300FFF1FB0
:10BAF000440FFF1F580FFF1F6C0FFF1F1C0FFF1F6E
:10BB00001C0FFF1F1C0FFF1F08004000100020002B
:10BB100018006000280050003800700058006800CD
:10BB2000100000003CBB000808BB00080C0000002F
:10BB30002F002F002A00240020002100FF7F00009A
:10BB40004176FB30825A825AFB3041760000FF7FFB
:10BB500004CF41767DA5825ABE89FB30008000006B
:10BB6000BE8904CF7DA57DA504CFBE8990BB00080A
:10BB700000000020380200008436000830BC0008B5
:10BB80003802002028180000F6B10008000000006C
:10BB900001CC420413127A1A01021112021301AAF3
:10BBA0001280126612551249124012381233122FA7
:10BBB000122B122712251223122232FF135945424B
:10BBC0000832FE5AB50C414BBD440C32104B3D4679
:10BBD0000C32115A5518327A5AFD0C9A090C3270EF
:10BBE0004B41390C9A720C9A740C9A760C9A780C18
:10BBF0009A7B0C9A7D0C32714BE13F0C9A730C9A34
:10BC0000750C9A770C9A790C9A7C0C9A7E0C6A6562
:10BC1000E8124E7308611A510C726013F14D7308EB
:10BC200064132D4FA408FFFF32013204000000000E
:0400000508002CC102
:00000001FF
